:100000000C94B2070C94DA070C94DA070C94DA0714
:100010000C94DA070C94DA070C94DA070C94DA07DC
:100020000C94DA070C94DA070C946C190C94DB1915
:100030000C94DA070C94DA070C94DA070C94DA07BC
:100040000C94DA070C94DA070C94DA070C94DA07AC
:100050000C94DA070C94DA070C94DA070C940D1C54
:100060000C94DA070C94DA070C94DA070C94DA078C
:100070000C94DA070C94DA070C94DA070C94DA077C
:100080000C94DA070C94DA070C94DA070C94DA076C
:100090000C94DA070C94DA070C94DA070C94DA075C
:1000A0000C94DA070C94DA070C94DA0744617900AF
:1000B00041636374004C6F616E00436170616369FA
:1000C0007479200053707261792000050512151FA4
:1000D000150905082466E766244120596573202028
:1000E00042204E6F000043616E6479204361737457
:1000F0006C6500536F6461205377616D70004775C4
:100100006D6D7920466F726573740043686F636F1D
:100110006C616E640049636520437265616D2052B5
:1001200064005377656574205375697465730000C6
:100130004C6F6C6C7900536F757273004D61727304
:10014000004165726F004865727368657900502ED2
:100150005375676172002000200003081F051F1FF0
:10016000151B1F11111F110E1F15111F05011F1146
:100170001D1F041F001F0010101F1F041B1F101045
:100180001F061F1F011F1F111F1F05071F311F1FE4
:10019000051B17151D011F011F101F0F100F1F0C2E
:1001A0001F1B041B071C071915130C121E1F120C12
:1001B0001E12120C121F0C1A14041F052E2A1E1FC9
:1001C000021C001D00201D001F041A011F001E0438
:1001D0001E1E021E1E121E3E120C0C123E1E020697
:1001E00014120A020F121E101E0E100E1E081E1AE6
:1001F000041A2E281E1A12161F111F001F001D158B
:100200001711151F07041F17151D1F151D01011FAD
:100210001F151F17151F00170000100020100000E9
:10022000030004083E09093E3F25251A1E2121121C
:100230003F21211E3F2525213F0505011E21293A89
:100240003F04043F213F21001021211F3F040A31B8
:100250003F2020203F02023F3F02043F1E21211E7B
:100260003F0909061E21112E3F09093622252519AD
:10027000013F01011F20201F0F10201F3F10103FC2
:100280003B04043B03043807312D2321102A2A3C68
:100290003F2424181C2222141824243F1C2A2A2C10
:1002A000047E05014C52523E3F040438243D200098
:1002B0004040443D3F081422213F20003E04043EBC
:1002C0003E04023C1C22221C7E22221C1C22227E76
:1002D0003E040204242A2A12021F22201E20201E6D
:1002E0000E10201E3E10103E360808364E50503E6E
:1002F000322A26221E29251E223F200032292926A5
:100300001221251A0C0A3F08172525191E25251824
:10031000013905031A25251A0629291E002F000078
:10032000002000004020000000030000000000004A
:10033000003E5B4F5B3E3E6B4F6B3E1C3E7C3E1C6B
:10034000183C7E3C181C577D571C1C5E7F5E1C00B1
:10035000183C1800FFE7C3E7FF0018241800FFE768
:10036000DBE7FF30483A060E2629792926407F052B
:100370000507407F05253F5A3CE73C5A7F3E1C1C41
:1003800008081C1C3E7F14227F22145F5F005F5F01
:1003900006097F017F006689956A606060606094ED
:1003A000A2FFA29408047E040810207E20100808F2
:1003B0002A1C08081C2A08081E101010100C1E0CFD
:1003C0001E0C30383E3830060E3E0E06000000008F
:1003D0000000005F00000007000700147F147F1476
:1003E000242A7F2A122313086462364956205000BB
:1003F00008070300001C2241000041221C002A1CA7
:100400007F1C2A08083E0808008070300008080891
:100410000808000060600020100804023E514945B1
:100420003E00427F400072494949462141494D33CF
:100430001814127F1027454545393C4A4949314136
:10044000211109073649494936464949291E000004
:100450001400000040340000000814224114141459
:100460001414004122140802015909063E415D5945
:100470004E7C1211127C7F494949363E414141224E
:100480007F4141413E7F494949417F090909013E78
:10049000414151737F0808087F00417F410020409F
:1004A000413F017F081422417F404040407F021CB1
:1004B000027F7F0408107F3E4141413E7F090909C8
:1004C000063E4151215E7F09192946264949493294
:1004D00003017F01033F4040403F1F2040201F3F5A
:1004E0004038403F631408146303047804036159DF
:1004F000494D43007F414141020408102000414121
:10050000417F0402010204404040404000030708CC
:100510000020545478407F284444383844444428C8
:10052000384444287F385454541800087E0902186F
:10053000A4A49C787F0804047800447D40002040F7
:10054000403D007F1028440000417F40007C04783B
:1005500004787C080404783844444438FC18242483
:100560001818242418FC7C08040408485454542403
:1005700004043F44243C4040207C1C2040201C3C80
:100580004030403C44281028444C9090907C446477
:10059000544C44000836410000007700000041360A
:1005A000080002010204023C2623263C1EA1A16190
:1005B000123A4040207A38545455592155557941C2
:1005C0002154547841215554784020545579400C99
:1005D0001E5272123955555559395454545939557A
:1005E0005454580000457C410002457D42000145BD
:1005F0007C40F0292429F0F0282528F07C5455452A
:10060000002054547C547C0A097F493249494932BC
:100610003248484832324A4848303A4141217A3AD1
:1006200042402078009DA0A07D39444444393D409B
:1006300040403D3C24FF2424487E4943662B2FFC48
:100640002F2BFF0929F620C0887E090320545479F6
:10065000410000447D413048484A32384040227AC7
:10066000007A0A0A727D0D19317D2629292F282644
:100670002929292630484D4020380808080808084C
:100680000808382F10C8ACBA2F102834FA00007BA5
:10069000000008142A142222142A140895002200AB
:1006A00095AA005500AAAA55AA55AA000000FF0065
:1006B000101010FF00141414FF001010FF00FF10A2
:1006C00010F010F0141414FC001414F700FF0000D4
:1006D000FF00FF1414F404FC141417101F10101F53
:1006E000101F1414141F00101010F0000000001F41
:1006F000101010101F10101010F010000000FF104C
:100700001010101010101010FF10000000FF140047
:1007100000FF00FF00001F10170000FC04F4141479
:100720001710171414F404F40000FF00F714141445
:1007300014141414F700F7141414171410101F10C5
:100740001F141414F4141010F010F000001F101FE8
:100750000000001F14000000FC140000F010F01056
:1007600010FF10FF141414FF141010101F000000CD
:1007700000F010FFFFFFFFFFF0F0F0F0F0FFFFFFD1
:100780000000000000FFFF0F0F0F0F0F3844443828
:10079000447C2A2A3E147E02020606027E027E0263
:1007A00063554941633844443C04407E201E200682
:1007B000027E020299A5E7A5991C2A492A1C4C72BF
:1007C00001724C304A4D4D303048784830BC625A46
:1007D000463D3E494949007E0101017E2A2A2A2AD6
:1007E0002A44445F444440514A444040444A5140B2
:1007F0000000FF0103E080FF000008086B6B083673
:1008000012362436060F090F0600001818000000E3
:100810001010003040FF0101001F01011E00191DD2
:100820001712003C3C3C3C0000000000D5F08D1449
:10083000A1C881CFD9F1AF2000F0F89C8E878387C3
:100840008E9CF8F00000FEFF0303030303070EFC79
:10085000F80000FEFF0303030303070EFCF800008B
:10086000FFFF00000000000000FFFF0000FEFF830C
:1008700083838383C7EE7C380000F8FC0E070303F4
:1008800003070EFCF800003F7FE0C08080C0E07FDF
:100890003FFFFF01010101010101FFFF0000FFFF18
:1008A0000C0C0C0C1C3E77E3C100007FFFC0C0C0E5
:1008B000C0C0E0703F1F00001F3F70E0C0C0C0E03C
:1008C000703F1F00007FFFC1C1C1C1C1E3773E1C63
:1008D00000001F3F70E0C0C0C0E0703F1F0000007C
:1008E000000001FFFF01000000647572696E67205F
:1008F0007468652063686173652121006275636BAC
:10090000732066726F6D2070757273657300596F16
:100910007520736E6174636865642000546865793E
:1009200020616C6C20676176652075702100412024
:100930004D6F6D2067617665207570212100002064
:1009400020596F75206D6973736564212121000042
:100950006861766520746F2072756E2100616E7912
:100960002073707261792120596F7500596F75205D
:10097000646F6E27742068617665007468656D2108
:1009800000596F752063616E2774207368616B6511
:1009900000616E20616C6C6579212100596F7520B2
:1009A0006C6F7374207468656D20696E00756E6974
:1009B0007473206F663A2000596F7520666F756EEC
:1009C000642000323030206275636B733F006D6FBE
:1009D000726520737061636520666F720063616E7B
:1009E0006479207361636B20776974680057696C60
:1009F0006C20796F75206275792061206E657700B3
:100A000057696C6C20796F75206561742069743F3B
:100A1000006D6F73746C7920756E636865776564BB
:100A2000212100686572652074686174206C6F6FA5
:100A30006B73005468657265277320736F6D652052
:100A400067756D00646F6C6C6172733F00737072D8
:100A5000617920666F7220343030004D6F6D2072E6
:100A60006570656C6C616E74007374696E6B207375
:100A70007072617920666F7200736C6565702073A7
:100A80007072617920666F720034303020646F6C50
:100A90006C6172733F0057696C6C20796F752062CE
:100AA0007579206100616674657220796F75210027
:100AB000667269656E64732061726500206F6620DE
:100AC00068657200616E642000596F7572204D6F09
:100AD0007468657200746F2063686172697479214B
:100AE00000596F7520676176652061206269740026
:100AF000617265206F7574726167656F757321210E
:100B000021210073686F72746167652120507269DA
:100B100063657300506F77646572656420737567F1
:100B20006172007072696365732121210061742014
:100B30006F7574726167656F757300627579696E40
:100B40006720486572736865790043686F636F68F2
:100B50006F6C696373206172650062616B652D6FF4
:100B60006666212121210066726F6D206C617374AD
:100B7000207765656B277300636865617020486541
:100B80007273686579004D6F6D73206172652073B3
:100B9000656C6C696E6700626F74746F6D6564205C
:100BA0006F7574212121004D617273207072696329
:100BB00065732068617665006C6F6C6C792121210A
:100BC000006172652073656C6C696E67206368658F
:100BD0006170004B696473206174207363686F6F88
:100BE0006C00746F6461792100626F72726F776557
:100BF00064206D6F6E657900596F7520616C726548
:100C0000616479002100596F7520646F6E2774202C
:100C10006861766520616E7900004F6F7073210006
:100C20002100596F752063616E2774206166666FBD
:100C3000726400004F6F7073210021006D6F726548
:100C40002000596F752063616E2774206361727292
:100C50007900004F6F70732100596F7527726520FE
:100C60006361756768742121006265656E2068693B
:100C7000742100596F75277665006D69737365641B
:100C80002121005468657900796F75212120005475
:100C9000686579277265206E616767696E670041D4
:100CA0002053707261792020422052756E004552A7
:100CB000524F522000416D7400536176696E677324
:100CC00000596F75206F776500596F7520686176E0
:100CD00065005769746864726177204D6F6E65793D
:100CE000004465706F736974204D6F6E65790042C2
:100CF0006F72726F77204D6F6E6579005061792049
:100D00004C6F616E00000051747900507269636528
:100D100000436F73747300596F75206861766500C6
:100D200053656C6C200042757920000000796F7566
:100D3000722074656574683F0064656E74697374CD
:100D400020746F2066697800646F6C6C6172732028
:100D5000666F7220610057696C6C20796F75207026
:100D60006179203130303000596F757220686561CB
:100D70006C74683A20007374696C6C2061667465E9
:100D80007220796F752100204D6F6D730054686576
:100D900072652061726520004265696E6720636834
:100DA00061736564212100576974686472617720FA
:100DB0004D6F6E6579004465706F736974204D6F77
:100DC0006E65790042616E6B00426F72726F7720C0
:100DD0004D6F6E6579005265706179204C6F616E60
:100DE0000052696368204275646479004A65742022
:100DF00066726F6D200053656C6C2043616E647980
:100E0000004275792043616E64790043616E6479B4
:100E1000205361636B0042616E6B0052696368200E
:100E20004275646479004A65740043616E64792098
:100E30005361636B0053656C6C2043616E64790091
:100E40004275792043616E64790048697420746842
:100E500065205374726565747321210076312E30DC
:100E60002E310043616E6479576172001E1E0000CE
:100E70000000000000000000000000C0F0E8C48294
:100E800002033F3F0F8782C2C4C8F0C000000000C9
:100E90000000008080807088A80FF1810181C1E18D
:100EA000F0FCF000818143271F0700000000008054
:100EB00040A1562C1434224176080D090701010186
:100EC00001010000000000003028140A05020100A2
:100ED0000000000000000000000000000000000012
:100EE000000000000000080B0002020200000904DC
:100EF0000000010202000005240010010524010188
:100F000001042402060524060001070581031000E0
:100F10004009040100020A00000007050202400027
:100F200000070583024000000403090412010002C7
:100F3000EF020140412336800001010203014172AA
:100F40006475696E6F204C4C430041726475696E24
:100F50006F204C656F6E6172646F0003051F0E0495
:100F60008A1CCB2E11241FBECFEFDAE0DEBFCDBF2F
:100F700012E0A0E0B1E0E6E5FBE602C005900D92CC
:100F8000A635B107D9F727E0A6E5B2E001C01D926A
:100F9000A03AB207E1F717E0C1EBD7E004C0219710
:100FA000FE010E94A633C03BD107C9F70E940B1D6A
:100FB0000C949E350C940000E6EEF2E0A0E0B8E060
:100FC00000800EBC8111012C1197A0FDFDCF019274
:100FD000B9F70DB40895480F592F511D1416150671
:100FE00084F5803891056CF597FF02C090E080E0B1
:100FF0004138510514F040E850E0481BFB01E77010
:10100000FF2721E001C0220FEA95EAF777FF02C02F
:10101000695F7F4FFB0133E0F595E7953A95E1F77E
:10102000F695FE2FEE27F795E795E80FF91FEA51A1
:10103000FD4F415030F08191DF011197822B8C934D
:10104000F8CF08956F927F928F929F92AF92BF9246
:10105000CF92DF92EF92FF920F931F93CF93DF9384
:10106000DC01FA011491319654913196C12FD0E0F0
:10107000222309F1CC24C394D12C852F877011F43D
:10108000D12CC12CE52EE694E694E694EC0CFD2CD4
:10109000F11CEC9EC001ED9E900DFC9E900D112464
:1010A000033011F4880F991F289F7001299FF00CBD
:1010B0001124EE0DFF1D7D01EC0EFD1E1E141F04FC
:1010C0000CF06BC0A038B1050CF067C0CB01850FE8
:1010D000911D181619060CF060C0603471050CF0F3
:1010E0005CC0309709F459C0362F3770CB0177FDBB
:1010F000079623E0959587952A95E1F7282F77FFA6
:1011000004C0332311F02FEF280F662777276A1BBF
:101110007B0BB7FD02C070E060E090E89A1B40E8EE
:10112000E416F1040CF4912F961BE22E022E000C13
:10113000FF08DE2CD0942F3F0CF0D12C41E0852FFE
:10114000877009F440E0B52EB694B694B6944B0D72
:10115000E40EF11C89E0E816F10414F048E0421BAB
:10116000B42EBD182D0D40E8240370011124AE0DDE
:10117000BF1DA60FB71F1D9D600D711D1124AF016E
:10118000460F571FC32E032E000CDD08033009F451
:10119000C7C090F4023009F474C0DF91CF911F9161
:1011A0000F91FF90EF90DF90CF90BF90AF909F9006
:1011B0008F907F906F9008950A3FA1F1B20E0B3F80
:1011C00061F72B1551F3BD016A517D4F10E000E02E
:1011D000091708F09FC0FA01E00FF11FE491F0E059
:1011E0004F010C2C02C0880C991C0A94E2F727FDD1
:1011F00006C0FB018081F82CF0948F21808333237B
:1012000061F0273054F47B01F0E8EF0EF11CA92CBB
:10121000A094F70180818A2180830F5F1F4F6F5F49
:101220007F4FD6CFB20E2B1509F4B7CFBD016A514F
:101230007D4F10E000E0091708F066C0FA01E00FEA
:10124000F11FE491F0E04F010C2C02C0880C991CB6
:101250000A94E2F727FD04C0FB018081882980837E
:10126000332351F0273044F47B01F0E8EF0EF11CFA
:10127000F7018081892980830F5F1F4F6F5F7F4F48
:10128000DACF6FEF70E0032E02C0660F771F0A946B
:10129000E2F760957095972E8B2C820E281509F435
:1012A0007CCF8D010A511D4FF12CE12CE91630F550
:1012B000FA01EE0DFF1DE491F0E03F010C2C02C09D
:1012C000660C771C0A94E2F727FD05C0F8018081BF
:1012D000862386298083332359F027304CF4580124
:1012E000F0E8AF0EB11CF501808189218729808348
:1012F000FFEFEF1AFF0A0F5F1F4FD8CF2F5F4C0F82
:101300005D1FA058BF4FCACF2F5F4C0F5D1FA05865
:10131000BF4F89CF2F5F4C0F5D1FA058BF4F51CFDC
:10132000E92EF12CFA01E60FF71FAA51BD4F60E834
:1013300070E06E197F09CE19DF098E01000F111FB1
:1013400041E050E07A01032E01C0EE0C0A94EAF766
:10135000592F4B2D892E932ECF93DF93ED01EF96CE
:10136000EF962296A590C590992059F0AE9C500119
:10137000CE9C600127302CF4F880D094FD20FB280F
:10138000F99222233AF0FC90C094FC20FA28FD92B6
:101390000C94CB0911965A9529F74A9551F0582D7E
:1013A00023951124E00FF11DA60FB11DC60FD11D0D
:1013B000D9CFDF91CF911124F0CE0F9302E020E03E
:1013C0000E9422080F9108952F923F924F925F92B0
:1013D0006F927F928F929F92AF92BF92CF92DF9245
:1013E000EF92FF920F931F93CF93DF93CDB7DEB7AA
:1013F00028970FB6F894DEBF0FBECDBF6F836A018A
:1014000019011C830B83FE82ED82811128C005E047
:1014100010E029E030E03A832983B6010D2C000C5E
:10142000880B990B0E940A304B015C015F815111BE
:101430001DC0E4E5F7E090E080E018861F828C157F
:101440009D050CF02BC1248135814F8158854217B1
:10145000530714F438872F8301963696F0CF04E0B3
:1014600010E048E050E05A834983D7CF20E030E0D5
:1014700040E05FE30E9469304B015C0120E030E016
:10148000A9010E94443320E030E040E05FE387FDA3
:1014900030C0C501B4010E94D8310E94B6327887AD
:1014A0006F83A6018F819885481B590BE4E5F7E00F
:1014B00090E080E0B12CA12C2F8138858217930712
:1014C000ECF086E0829FF001839FF00D1124EC5A2E
:1014D000F84F90E080E0D12CC12C84179507BCF424
:1014E00024813581C216D3060CF469010196369623
:1014F000F4CFC501B4010E94D731CFCF248135810B
:10150000A216B3060CF4590101963696D5CFB80150
:10151000110F880B990B0E940A302B013C01B50179
:101520006C0D7D1D072E000C880B990B0E940A3054
:1015300020E030E040EE5FE30E94D8316B017C0197
:1015400020E030E040E05FE3C301B2010E94693077
:101550009B01AC01C701B6010E9469306B017C019F
:1015600020E030E0A9010E94443320E030E040E078
:101570005FE387FD89C0C701B6010E94D8310E9490
:10158000B63202E410E0061B170BF1011183008351
:10159000B501BB0C880B990B0E940A3020E030E0AB
:1015A00040EE5FE30E94D831A30192010E946930AE
:1015B0004B015C0120E030E0A9010E94443320E0AF
:1015C00030E040E05FE387FD64C0C501B4010E94E4
:1015D000D8310E94B632600F711FEB81FC8171839C
:1015E000608329813A81B901330F880B990B0E94DE
:1015F0000A3020E030E040E05FE30E9469306B0198
:101600007C014F815885BA01550F880B990B0E94B8
:101610000A309B01AC01C701B6010E9469306B0121
:101620007C0120E030E0A9010E94443320E030E05A
:1016300040E05FE387FD85C0C701B6010E94D83155
:101640000E94B6322AE230E0C901861B970BED8179
:10165000FE819183808328960FB6F894DEBF0FBE7B
:10166000CDBFDF91CF911F910F91FF90EF90DF9051
:10167000CF90BF90AF909F908F907F906F905F9032
:101680004F903F902F900895C701B6010E94D73127
:1016900076CFC501B4010E94D7319BCFB801110F9D
:1016A000880B990B0E940A3020E030E040E05FE3B5
:1016B0000E9469302B013C01EF81F885BF01FF0FCB
:1016C000880B990B0E940A309B01AC01C301B20147
:1016D0000E9469302B013C0120E030E0A9010E940A
:1016E000443320E030E040E05FE387FD25C0C301E4
:1016F000B2010E94D8310E94B63222E430E0C90122
:10170000861B970BF101918380838FEF9FEFEB8115
:10171000FC819183808329813A81B901330F880B41
:10172000990B0E940A3020E030E040E05FE30E9425
:101730006930A501940171CFC301B2010E94D73174
:10174000DACFC701B6010E94D7317ACFFC01809170
:10175000E502882311F13FB7F89482E08093E90015
:101760002091F200822F90E01816190614F481E0FF
:1017700090E0882339F0289844E64093E4024091B1
:10178000F1004083222339F02091F200211103C09F
:101790002BE62093E8003FBF08958FEF9FEF089559
:1017A0002FB7F89483E08093E9009091E800892FA7
:1017B000807295FF04C09091F20080E4891B2FBFD6
:1017C00008958091DC0281110DC082E08093D802DF
:1017D00084E08093D9021092DB021092DA0281E059
:1017E0008093DC0288ED92E00895CF93DF931F92FF
:1017F000CDB7DEB76983DC01ED91FC910280F38106
:10180000E02D41E050E0BE016F5F7F4F09950F90E2
:10181000DF91CF91089583E08093E9008091F200F9
:10182000882319F08AE38093E80008950E94D00B82
:1018300090E00895CF93DF931F92CDB7DEB7FC0100
:101840008485958597FD08C02FEF3FEF3587248766
:101850000F90DF91CF910895CE0101960E94A60BC3
:10186000019719F4898190E0F3CF8FEF9FEFF0CFCC
:101870000F931F93CF93DF931F92CDB7DEB78C01E9
:10188000FC018485958597FF0BC0CE0101960E94CF
:10189000A60B019771F4898190E0F8019587848700
:1018A000F801848595850F90DF91CF911F910F915D
:1018B00008958FEF9FEFF1CFFC018485958597FD0B
:1018C0000BC09FB7F89482E08093E9008091F2000A
:1018D0009FBF90E0019608959FB7F89482E08093AF
:1018E000E9008091F2009FBF90E008954091D202FC
:1018F0005091D3022091D0023091D1024217530768
:10190000B4F49091E8009570E1F39091E80092FDB5
:1019100019C08093F1008091D2029091D302019678
:101920008F739927892B19F48EEF8093E8008091AB
:10193000D2029091D30201969093D3028093D20267
:1019400081E0089580E00895DF92EF92FF920F9377
:101950001F93CF93DF93D82E8A01EB017B01E40E16
:10196000F51ECE15DF0559F0D7FE12C0FE01849199
:101970000E94760C21968111F4CF0FEF1FEFC80162
:10198000DF91CF911F910F91FF90EF90DF9008951D
:101990008881EECF0F931F93CF93DF931F92CDB724
:1019A000DEB782E0898342E450E066EE7EE080E8C4
:1019B0000E94A40C0E94E10BDC0112960D911C9177
:1019C0000115110589F0D801ED91FC910280F38198
:1019D000E02DBE016F5F7F4FC801099597FD04C0E0
:1019E000F80100851185ECCF89810F90DF91CF91AF
:1019F0001F910F910895615030F02091F100FC018A
:101A000020830196F8CF289884E68093E402089515
:101A10003FB7F8948091CC029091CD02A091CE0274
:101A2000B091CF0226B5A89B05C02F3F19F00196B3
:101A3000A11DB11D3FBFBA2FA92F982F8827BC0128
:101A4000CD01620F711D811D911D42E0660F771F50
:101A5000881F991F4A95D1F708958F929F92AF9250
:101A6000BF92CF92DF92EF92FF926B017C010E94B6
:101A7000080D4B015C01C114D104E104F104B9F07B
:101A80000E94080D681979098A099B09683E73400C
:101A90008105910580F321E0C21AD108E108F1081F
:101AA00088EE880E83E0981EA11CB11CE4CFFF9045
:101AB000EF90DF90CF90BF90AF909F908F90089560
:101AC0008F929F92AF92BF92CF92DF92EF92FF924E
:101AD0000F931F93CF93DF936C017B018A01809159
:101AE0000C01882309F45CC08091E502882309F485
:101AF00057C08091D70280FF05C08091E0008260CE
:101B00008093E000E801B12C8AEFA82E93E0892EA3
:101B10002AE3922E209711F4BB20D9F10E94D00B1A
:101B200081110AC0AA94AA20D9F161E070E080E096
:101B300090E00E942D0DEECF8C171D0611F00CF0D9
:101B40008C2F9FB7F8948092E9002091E80025FD42
:101B500002C09FBFDFCF282F30E0C21BD30BF7019D
:101B6000815020F041914093F100FACFE20EF31E34
:101B7000BB2021F09092E800B12CEBCF8091E800DF
:101B800085FDE7CF9092E800BB24B394209709F33A
:101B9000F3CF5D9884E68093D602101611063CF0D0
:101BA00081E090E0F6019383828310E000E0C801B9
:101BB000DF91CF911F910F91FF90EF90DF90CF9029
:101BC000BF90AF909F908F9008950895DB01149679
:101BD0004D915C9115976D917C91DC01ED91FC919B
:101BE0000280F381E02D09942F923F924F925F92F1
:101BF0006F927F928F929F92AF92BF92CF92DF921D
:101C0000EF92FF920F931F93CF93DF9300D000D0FA
:101C100000D0CDB7DEB7782E662E5A0128E0422ECE
:101C2000512C811103C099E0492E512CCE0101960F
:101C30007C018E010D5F1F4F9E012B5F3F4FA50161
:101C4000662D872D0E94E409B5010B2C000C880B32
:101C5000990B0E940A3020E030E040E05FE30E94F0
:101C600069306B017C0120E030E0A9010E9444331F
:101C700020E030E040E05FE387FD24C0C701B6010B
:101C80000E94D8310E94B6328B0184E5C82E87E0CD
:101C9000D82E049D1001059D300C149D300C11248C
:101CA000F12CE12C912C812C8A149B04B4F58981B0
:101CB0009A81662019F0801691064CF42D818E0DC4
:101CC0009F1D0BC0C701B6010E94D731DBCF2B810E
:101CD000A70142195309840F951F7720A1F0209383
:101CE00089072093880780938A07B60184E897E0E4
:101CF0000E94E60D9FEF891A990A86E0C80ED11C52
:101D0000E40CF51CD1CF2093930720939207809386
:101D10009407B6018EE897E0EBCF26960FB6F894BD
:101D2000DEBF0FBECDBFDF91CF911F910F91FF900E
:101D3000EF90DF90CF90BF90AF909F908F907F906B
:101D40006F905F904F903F902F900895EF92FF9289
:101D50000F931F93CF93DF938C017B01D0E0C0E002
:101D6000F701EC0FFD1F6491662361F0D801ED913E
:101D7000FC910190F081E02DC8010995892B11F0AB
:101D80002196EECFCE01DF91CF911F910F91FF9061
:101D9000EF900895AF92BF92CF92DF92EF92FF92B1
:101DA0000F931F93CF93DF936C017B018B01040F83
:101DB000151FEB015E01AE18BF08C017D10759F01F
:101DC0006991D601ED91FC910190F081E02DC60161
:101DD0000995892B79F7C501DF91CF911F910F915B
:101DE000FF90EF90DF90CF90BF90AF9008952D9A25
:101DF0000895BC0190E080E00C942D0D8FB180958A
:101E0000807F669B88601C9B8460089581EC809332
:101E10007C0085B1806F85B984B1877E84B984B137
:101E2000876E84B95E9A5F988AB1806D8AB9769A16
:101E30006E9881B3806F81BB899880B38D7080BBB1
:101E400080E58CBD81E08DBD85E090E00E94F90EBB
:101E50005F9A85E090E00E94F90E5E985C98ECE253
:101E6000F8E084918EBD00000DB407FEFDCF3196E1
:101E700088E0E933F807A9F75C9A81E88093640069
:101E800080916500816080936500089590915E0265
:101E9000982329F490915F02982381E009F480E06F
:101EA0000895CF93C82F0E94FE0E982F9C2381E0A7
:101EB0009C1380E0CF91089580E00C94DC0780387B
:101EC0009105B8F460347105A0F420E191E061FD62
:101ED00094E060FD990F62FD9295687F269FD00186
:101EE0001124A80FAA51BD4F8C9140FF03C0892B2C
:101EF0008C93089590958923FBCF2F923F924F9218
:101F00005F926F927F928F929F92AF92BF92CF9289
:101F1000DF92EF92FF920F931F93CF93DF937C0199
:101F20006B0188248394912CD0E0C0E005E010E0A0
:101F300096EF692E77247A942CEFA22EBB24BA94C4
:101F4000842F8470582E842F8270482E842F88709E
:101F5000382E4170242E219682E0880E911CA80C08
:101F6000B91C552091F041E0B8016C0D7D1DC701F1
:101F70008C0F9D1F0E945F0F41E0B6016C0F7D1F0B
:101F8000C8018E0D9F1D0E945F0F442091F041E01B
:101F9000B601601B710BC7018C0F9D1F0E945F0F64
:101FA00041E0B6016C1B7D0BC8018E0D9F1D0E9488
:101FB0005F0F332091F041E0B6016C0F7D1FC70128
:101FC000801B910B0E945F0F41E0B8016C0D7D1DDD
:101FD000C7018C1B9D0B0E945F0F222091F041E0F6
:101FE000B6016C1B7D0BC701801B910B0E945F0F1C
:101FF00041E0B601601B710BC7018C1B9D0B0E9459
:102000005F0FC017D10754F4B7FCA5CF01501109D9
:1020100082E0680E711CA60CB71C9DCFDF91CF919A
:102020001F910F91FF90EF90DF90CF90BF90AF90F6
:102030009F908F907F906F905F904F903F902F90E8
:1020400008952F923F924F925F926F927F928F925C
:102050009F92AF92BF92CF92DF92EF92FF920F9337
:102060001F93CF93DF93EC0141E06FE370E00E9498
:102070005F0F41E065E370E0CE010E945F0F41E039
:102080006AE370E0CE0105960E945F0F41E06AE3CB
:1020900070E0CE0105970E945F0F22242394312C1B
:1020A000F12CE12C05E010E036EF432E55245A9434
:1020B0004CEFC42EDD24DA948FEFE81AF80A82E0A0
:1020C000280E311CC20CD31C47018C0E9D1E41E012
:1020D00058018AE3A80EB11CB501C4010E945F0F2C
:1020E0003E016E187F0841E0B501C3010E945F0FF9
:1020F00041E08AE3A82EB12CA01AB10AB501C401AF
:102100000E945F0F41E0B501C3010E945F0F4701CC
:102110008AE3880E911C41E0B4015E01A00EB11E5D
:10212000C5010E945F0F41E0B4013E01601A710ACF
:10213000C3010E945F0F9AE3892E912C8E189F088D
:1021400041E0B401C5010E945F0F41E0B401C30149
:102150000E945F0FE016F1069CF0DF91CF911F9176
:102160000F91FF90EF90DF90CF90BF90AF909F9036
:102170008F907F906F905F904F903F902F90089539
:10218000D7FC9ACF0150110982E0480E511CC40CB3
:10219000D51C92CF8F929F92AF92BF92CF92DF9237
:1021A000EF92FF920F931F93CF93DF936D3089F0DF
:1021B000C0905C02D0905D026A30D1F410925B0254
:1021C00010925A0288E0C80ED11CD0925D02C092D3
:1021D0005C0281E090E0DF91CF911F910F91FF9021
:1021E000EF90DF90CF90BF90AF909F908F90089529
:1021F00000915A0210915B02E5E06E9FE00111240C
:10220000C45DDC4F4801F12CF5E0E12CFF1629F00C
:10221000CE010196FE01E490EC01B12CA12C4E2DD3
:102220004170B6016A0D7B1DC4010E945F0FE694E8
:10223000FFEFAF1ABF0A88E0A816B10481F7F39444
:10224000EFEF8E1A9E0AF6E0FF12DECF0A5F1F4FF5
:1022500010935B0200935A02BCCFDF92EF92FF9281
:102260000F931F93CF93DF937C01D22E8B01040F2A
:10227000111DEB0177FF02C0D0E0C0E0C8010134BE
:10228000110514F080E490E0C817D9073CF44D2DF7
:10229000BE01C7010E945F0F2196F0CFDF91CF9161
:1022A0001F910F91FF90EF90DF9008952F923F9232
:1022B0004F925F926F927F928F929F92AF92BF9256
:1022C000CF92DF92EF92FF920F931F93CF93DF9302
:1022D00000D000D000D0CDB7DEB76C01762E542EE2
:1022E0004901602E98E0A92EB12C611103C089E04C
:1022F000A82EB12CCE0101967C018E010D5F1F4FDF
:102300009E012B5F3F4FA401652D872D0E94E4099C
:1023100009811A81552011F1B401990C880B990B90
:102320000E940A3020E030E040E05FE30E94693024
:102330001B012C0120E030E0A9010E94443320E081
:1023400030E040E05FE387FD0CC0C201B1010E94B4
:10235000D8310E94B632C616D70644F48D809E80CE
:1023600009C0C201B1010E94D731F3CF8B809C809C
:10237000C61AD70ACA9CB001CB9C700DDA9C700DAE
:102380001124060F171FC40104976620B1F061E005
:1023900070E0711002C062E070E0060F171F6C0160
:1023A000C6012FEFC21AD20AC814D90491F020E056
:1023B00045E0B8010E942D11F3CF61E070E071108B
:1023C00002C062E070E0600F711F4BE55FE00E94A9
:1023D000DD0926960FB6F894DEBF0FBECDBFDF91A4
:1023E000CF911F910F91FF90EF90DF90CF90BF9012
:1023F000AF909F908F907F906F905F904F903F90A5
:102400002F9008950F93CF93DF93EC019E816A3054
:1024100059F48D818C836985960F9E8381E090E0CD
:10242000DF91CF910F910895262F61E0690F2A3334
:1024300098F4203378F5273249F140F4213261F1E4
:1024400098859C5F8C81890F8C83E8CF2C3231F189
:102450002E32B1F72FE309C0213490F32B35C0F0B1
:102460008FE9820F27548A3158F7062E000C770B1C
:102470008C81082E000C990B3F810AEF313009F056
:102480000BEF42E252E00E942208DACF21E4EDCFC6
:102490002154EBCF2C5FE9CF2EE3E7CF20E4E5CF4B
:1024A0000F93CF93DF93EC019E816A3059F48D81B5
:1024B0008C836985960F9E8381E090E0DF91CF91B8
:1024C0000F910895262F61E0690F2A3398F4203385
:1024D00078F5273249F140F4213261F198859D5F0A
:1024E0008C81890F8C83E8CF2C3231F12E32B1F7F9
:1024F0002FE309C0213490F32B35C0F08FE9820F10
:1025000027548A3158F7062E000C770B8C81082E41
:10251000000C990B3F810AEF313009F00BEF4AE5CF
:1025200051E00E942208DACF21E4EDCF2154EBCF15
:102530002C5FE9CF2EE3E7CF20E4E5CFE2EAF2E03B
:102540008AEB92E030E020E04191519161917191EC
:10255000240F351F8E179F07B9F780916F02909156
:102560007002821B930B0895CF93C82F84E00E94C2
:10257000460F811107C0CC2381F088E00E94460FEE
:10258000882359F01092C6028091810290918202B4
:102590009093C3028093C20281E0CF910895E4E852
:1025A000F7E08AE48583848387E3868369ED70E0BE
:1025B000CF010E94A60E8BE490E00E94211087E6D6
:1025C00090E00C942110CF92DF92EF92FF920F9344
:1025D0001F93CF93DF9346E770E060E085E090E0E3
:1025E0000E94EB0746E76FE370E085E090E00E9411
:1025F000EB0721E046E365E070E090E080E00E94B8
:102600002D1121E046E365E070E08FE790E00E9445
:102610002D1141E065E070E085E090E00E947D0FC3
:1026200042E065E070E08AE790E00E947D0F44E0C0
:102630006AE370E08AE790E00E947D0F48E06AE379
:1026400070E085E090E00E947D0F80918302C6E3F8
:10265000D7E0811122C00AE010E0F12CE12C8AE0E1
:10266000C82ED12C8091840290918502E816F9063B
:1026700084F58FEFE81AF80AD0925B02C0925A02F2
:1026800010935D0200935C02BE0188E997E00E940E
:10269000E60D065F1F4F2696E5CF1AE0F12CE12CE0
:1026A0000AE08091840290918502E816F9068CF484
:1026B000009393070093920710939407BE018EE84E
:1026C00097E00E94E60D8FEFE81AF80A175F26964A
:1026D000E8CFDF91CF911F910F91FF90EF90DF90A6
:1026E000CF900895BC01EEE8F7E096E095839483DF
:1026F0008CE08683CF010C94E60D90E080E0089595
:102700008F929F92AF92BF92EF92FF920F931F937F
:10271000CF93DF93CDB7DEB7A1970FB6F894DEBFA6
:102720000FBECDBF7C01FA01CB0119A2223008F403
:102730002AE08E010F5D1F4F822E912CB12CA12C0F
:10274000BF01A50194010E94A631F901CA016A30B6
:1027500074F5605DD8016E938D01232B242B252BFE
:1027600079F790E080E0109789F0FD01019000205A
:10277000E9F73197AF014A1B5B0BD701ED91FC9153
:102780000280F381E02DB801C7010995A1960FB62B
:10279000F894DEBF0FBECDBFDF91CF911F910F9197
:1027A000FF90EF90BF90AF909F908F900895695CDD
:1027B000D1CFCF92DF92EF92FF920F931F93CF93DF
:1027C000DF9377FF21C06A017B01EC01E881F98189
:1027D0000190F081E02D6DE209958C014427552789
:1027E000BA014C195D096E097F092AE0CE010E94E9
:1027F0008013800F911FDF91CF911F910F91FF9058
:10280000EF90DF90CF9008952AE0DF91CF911F9154
:102810000F91FF90EF90DF90CF900C948013CF93A7
:10282000DF93CFE1D0E020E04AE067E170E0CE0145
:102830000E942D112196CF36D105A9F783E280930E
:1028400093078093920788E18093940740916B02ED
:1028500050916C0260916D0270916E028EE897E06B
:10286000DF91CF910C94D913BC01EEE8F7E09AE028
:102870009583948388E18683CF010E94E60D48E525
:1028800066E170E08EE190E00E94EB0748E561E2CE
:1028900070E08EE190E00E94EB0721E04CE066E101
:1028A00070E08EE190E00E942D1121E04CE066E1A5
:1028B00070E085E790E00E942D110E940F1442ED18
:1028C00050E068E170E08FE690E00C94DD09CF9273
:1028D000DF92EF92FF920F931F93CF93C82F8B013C
:1028E00069017A016E5F7F4F4BEC50E00E94DD0979
:1028F000CA5FEEE8F7E0C583C4830683B701A6018B
:10290000CF01CF911F910F91FF90EF90DF90CF906B
:102910000C94D913CF93DF938091C2029091C3029C
:102920004197029768F5C8E2D0E020E047E065E211
:1029300070E0CE010E942D112196CF37D105A9F765
:10294000E0917F02F0918002EE0FFF1FEE0FFF1F5C
:10295000E657FD4F208131814281538160916B02A6
:1029600070916C0280916D0290916E020E9496337C
:102970009B01AC0165E270E088E290E00E94671480
:10298000DF91CF910C940F14CF93DF93EC018881EA
:102990009981009711F00E944834198218821D8293
:1029A0001C821B821A82DF91CF910895FC018081E5
:1029B0009181009711F00C9448340895CF93C82F5B
:1029C0008091C0029091C10201969093C1028093C0
:1029D000C00210926A020E943A2F21EE3EE240E0CD
:1029E00050E00E943D316058714C8F4F9F4F609373
:1029F0008A0270938B0280938C0290938D020E94C6
:102A00003A2F29E53BE140E050E00E943D31685714
:102A10007C4E8F4F9F4F60938E0270938F028093F6
:102A20009002909391020E943A2F23E230E040E01E
:102A300050E00E943D319B01AC01265F3F4F4F4F5C
:102A40005F4FA4E6B0E00E945C3160939202709305
:102A5000930280939402909395020E943A2F2BE266
:102A600030E040E050E00E943D319B01AC012F5D21
:102A70003F4F4F4F5F4FAAE0B0E00E945C31609340
:102A800096027093970280939802909399020E9405
:102A90003A2F20E130E040E050E00E943D319B01C0
:102AA000AC01295F3F4F4F4F5F4FAAE0B0E00E945B
:102AB0005C3160939A0270939B0280939C02909386
:102AC0009D020E943A2F25E030E040E050E00E9455
:102AD0003D319B01AC012F5F3F4F4F4F5F4FAAE04D
:102AE000B0E00E945C3160939E0270939F028093DD
:102AF000A0029093A102CC23C1F160917702709162
:102B000078028091790290917A020E940A302DEC2D
:102B10003CEC4CE85FE30E9469300E94EC320E947A
:102B2000B632609377027093780280937902909323
:102B30007A02609173027091740280917502909193
:102B400076020E940A3024E13EEA47E85FE30E94F1
:102B500069300E94EC320E94B63260937302709327
:102B6000740280937502909376021092C602CF9100
:102B700008950C9427310F931F93CF93DF938C010B
:102B8000EB01FC01808191810097E1F068817981FE
:102B900061157105A9F0428153812C813D81421755
:102BA000530770F00E9497358C819D81F8019583C1
:102BB00084831D821C82DF91CF911F910F91089514
:102BC0000E94483488819981F801918380838A81A9
:102BD0009B81938382838C819D81958384831982D9
:102BE00018821B821A82E5CF0F931F93CF93DF9336
:102BF000EC0188819981009759F02A813B81261741
:102C0000370730F081E0DF91CF911F910F91089548
:102C10008B016F5F7F4F0E94D134009759F09983E9
:102C200088831B830A832C813D81232B59F7FC0168
:102C30001082E8CF80E0E7CFEF92FF920F931F93CF
:102C4000CF93DF93EC017B01CB010E94992F00977A
:102C5000A9F00C811D81080F191FB801CE010E9437
:102C6000F415882361F0288139818C819D81B70119
:102C7000820F931F0E94922F1D830C8381E0DF91AE
:102C8000CF911F910F91FF90EF900895EF92FF92D7
:102C90000F931F93CF93DF93FB01E080F180E1144A
:102CA000F10441F480E0DF91CF911F910F91FF90EB
:102CB000EF9008950481158101151105B1F0EC0123
:102CC0008C819D81080F191FB801CE010E94F41557
:102CD000882341F3288139818C819D81B701820F3E
:102CE000931F0E9497351D830C8381E0DCCFEF9208
:102CF000FF920F931F93CF93DF93EC018B0161152C
:102D0000710551F0CB010E94992F7C01BC01CE01CD
:102D10000E94F41581110BC0CE010E94C414CE0193
:102D2000DF91CF911F910F91FF90EF900895FD8259
:102D3000EC82B801888199810E94922FF0CFFC012A
:102D40001182108213821282158214820C947716DB
:102D5000CF93DF93EC016230710501F148F4611506
:102D6000710581F061307105B1F06FE271E00CC066
:102D700064307105C9F0A8F065307105B1F760E302
:102D800071E002C06EE471E0CE010E949F16CE0198
:102D9000DF91CF91089566E471E0F6CF61E471E0D0
:102DA000F3CF6CE371E0F0CF66E371E0EDCFCF934A
:102DB000DF93EC016230710501F148F46115710592
:102DC00081F061307105B1F065EE70E00CC06430E7
:102DD0007105C9F0A8F065307105B1F766EE70E0D5
:102DE00002C062E271E0CE010E949F16CE01DF9127
:102DF000CF91089565E171E0F6CF6BE071E0F3CF1C
:102E00006EEF70E0F0CF63EF70E0EDCFEF92FF92E6
:102E10000F931F93CF93DF93EC017B018A01BA01DB
:102E20000E94F41581110BC0CE010E94C414CE0182
:102E3000DF91CF911F910F91FF90EF9008951D8327
:102E40000C83B701888199810E949735F0CFFB01EF
:102E500001900020E9F73197AF01461B570B0C9406
:102E600006170F931F93CF93DF93CDB7DEB762970B
:102E70000FB6F894DEBF0FBECDBF8C01CB01F801B9
:102E80001182108213821282158214824AE0BE01DE
:102E90006F5F7F4F0E94A22FBE016F5F7F4FC801FF
:102EA0000E94271762960FB6F894DEBF0FBECDBF03
:102EB000DF91CF911F910F9108950F931F93CF939F
:102EC000DF93CDB7DEB7A2970FB6F894DEBF0FBE83
:102ED000CDBF8C01CB01BA01F8011182108213829F
:102EE0001282158214822AE0AE014F5F5F4F0E946A
:102EF000AD2FBE016F5F7F4FC8010E942717A296BA
:102F00000FB6F894DEBF0FBECDBFDF91CF911F91FA
:102F10000F9108952F923F924F925F926F927F92FE
:102F20008F929F92AF92BF92CF92DF92EF92FF92D9
:102F30000F931F93CF93DF93CDB7DEB762970FB692
:102F4000F894DEBF0FBECDBF2C019E012F5F3F4F17
:102F5000490139011C01D12CC12C10E000E0B12C39
:102F6000A12CF10141915191619171911F01CE010B
:102F70000D960E945D17E988FA88CE010D960E9491
:102F8000D614B601CE010D960E94A81689899A8999
:102F9000E80EF91EFFEFEF1AFF0AF301E192F1923A
:102FA0003F01CE010D960E94D614F3E0CF16D10456
:102FB0000CF03FC0AE14BF040CF457012FEFC21A3F
:102FC000D20A36E0C316D10461F684E5C82E87E044
:102FD000D82EF12CE12C150183E0E816F1040CF059
:102FE0001801B701CE010D960E94A816BE01635FBD
:102FF0007F4FC6010E94BB15CE010D960E94D614CC
:1030000068E571E0C6010E941C16712C612CF40168
:10301000808191819101281B390B6216730674F42B
:1030200066E571E0C6010E941C163FEF631A730A41
:10303000EECF0E151F0514F68701C0CFF2014191A6
:103040005191619171912F01CE010D960E945D17F2
:10305000BE01635F7F4FC6010E944616CE010D96EA
:103060000E94D614FFEFEF1AFF0A26E0C20ED11C11
:1030700032E0830E911C86E0E816F10409F0ABCF34
:10308000F092BF02E092BE0281E08093BC020A0D82
:103090001B1D073111050CF480E08093BD02629680
:1030A0000FB6F894DEBF0FBECDBFDF91CF911F9159
:1030B0000F91FF90EF90DF90CF90BF90AF909F90D7
:1030C0008F907F906F905F904F903F902F900895DA
:1030D000EF92FF920F931F93CF93DF9300D000D016
:1030E00000D0CDB7DEB78091C2029091C30209979C
:1030F00009F05EC00E949E128C01BC01CE010196B7
:103100000E943117ED80FE80CE0101960E94D614F8
:1031100081E0809389078093880710928A0764EC86
:1031200070E084E897E00E94A60E409171025091F1
:103130007202052E000C660B770B84E897E00E9464
:10314000D91387E190E08E199F09880F991F880F86
:10315000991F809389078093880710928A076AEBEA
:1031600070E084E897E00E94A60EA801110F660B9C
:10317000770B84E897E00E94D91310E000E021E08B
:1031800041E068E070E0C8010E942D110F5F1F4F01
:1031900000381105A1F726960FB6F894DEBF0FBED2
:1031A000CDBFDF91CF911F910F91FF90EF900895C8
:1031B00040917B0250917C0260917D0270917E0271
:1031C000CE0101960E945D17ED80FE80CE01019632
:1031D0000E94D61400E210E00E191F09000F111F03
:1031E000000F111F8091C2029091C3029C012550D3
:1031F00031092230310508F052C021E020938907BF
:103200002093880710928A0760EB70E0059711F40D
:1032100065EB70E084E897E00E94A60E4BEC50E06E
:1032200061E070E083E190E00E94DD0989E1809334
:1032300089078093880710928A078091C202909133
:10324000C302059719F54091770250917802609179
:10325000790270917A0284E897E00E94D9134BECCE
:1032600050E061E070E0C80106970E94DD0900931C
:1032700089070093880710928A0740917B0250913A
:103280007C0260917D0270917E0273CF4091730247
:10329000509174026091750270917602DCCF81E0EA
:1032A000809389078093880710928A076CEA70E000
:1032B00084E897E00E94A60E8EE0809389078093B1
:1032C000880710928A074091C0025091C102052ED2
:1032D000000C660B770BBFCF1F920F920FB60F92A9
:1032E00011248F939F938091E1009091E100937F4F
:1032F0009093E10083FF0FC01092E90091E090935A
:10330000EB001092EC0092E39093ED001092E50236
:1033100098E09093F00082FF22C093E09093E90040
:103320009091F200992319F09AE39093E80090911C
:10333000D602992341F09091D60291509093D602F3
:10334000911101C05D9A9091E402992341F090910E
:10335000E40291509093E402911101C0289A84FFF5
:1033600018C08091E2008E7E81608093E20080919F
:10337000E1008F7E8093E1008091D7028E7E806194
:103380008093D7029F918F910F900FBE0F901F9047
:10339000189580FFF7CF8091E2008E7E8061809348
:1033A000E2008091E1008E7E8093E1008091D7025F
:1033B0008E7E8160E5CF1F920F920FB60F9211247F
:1033C000CF92DF92EF92FF920F931F932F933F9331
:1033D0004F935F936F937F938F939F93AF93BF931D
:1033E000EF93FF93CF93DF93CDB7DEB76C97DEBF3C
:1033F000CDBF1092E9008091E80083FF25C068E00E
:10340000CE0145960E94FB0C82EF8093E8008D89E7
:1034100087FF39C09091E80090FFFCCF982F9076FD
:1034200009F034C19E894F89588D2F89F88C9111EC
:1034300031C0803861F58091D5028093F1001092FF
:10344000F1008EEF8093E8006C960FB6F894DEBF23
:103450000FBECDBFDF91CF91FF91EF91BF91AF91A3
:103460009F918F917F916F915F914F913F912F919C
:103470001F910F91FF90EF90DF90CF900F900FBEB4
:103480000F901F9018959EEF9093E800C7CF109271
:10349000F100D5CF913059F48111D3CF413051058E
:1034A00081F68091D5028D7F8093D502CACF93306B
:1034B00049F48111C6CF4130510519F68091D502EA
:1034C0008260F2CF953041F48091E80080FFFCCF1C
:1034D00020682093E300B5CF963009F0A9C00B8D8A
:1034E0001C8D22E01092E9001092D3021092D202B9
:1034F000F2122EC01092D1021092D0020E94CA0C79
:103500001F8299E09983FA8291E09E8390EA9887DE
:103510009AEF99872091D2023091D302275F3F4FD3
:103520003C832B838D831092E9001092D30210927A
:10353000D2021093D1020093D00249E050E0BE01C4
:103540006F5F7F4F80E00E94A40C0E94CA0C79CF6D
:103550001093D1020093D0020E94E10BDC0112967D
:103560000D911C910115110509F451C1D801ED917E
:10357000FC910480F581E02DBE016B5E7F4FC80198
:103580000995009709F03EC1F80100851185EACF41
:10359000F3E0FF120EC08F89882309F440C0823007
:1035A00061F440E860E18AE49FE00E94571C8111C9
:1035B00048CF81E28093EB0047CF813029F440E887
:1035C0006BE08EE39FE0F1CF833099F70E94E10B2F
:1035D000DC011296ED90FC908E010F5F1F4F680189
:1035E000E114F10479F0D701ED91FC910680F781A7
:1035F000E02DB801C7010995080F111DF701E084FE
:10360000F184EECFD8011C92F60101900020E9F779
:103610003197BF016C197D0940E0C601C6CF68E251
:103620007FE0FB01449150E080E80E94A40C09CFA8
:10363000973009F4BECF983021F481E08093F100F7
:1036400000CF993009F0FDCE837009F0B2CFE8E1E8
:10365000F1E081E031E096E32191222371F0809343
:10366000E9003093EB00DF0111972C912093EC00DF
:103670009093ED008F5F873079F78EE78093EA00B3
:103680001092EA008F898093E502DBCE8B8D9C8DB2
:103690001092E9001092D3021092D2029093D102BC
:1036A0008093D002898D811192C08E899D89913A33
:1036B00049F4813209F07DCF47E050E065E071E0E8
:1036C00080E0B3CF913209F074CF833269F48F89EF
:1036D000988DB0E0A0E08093010190930201A09347
:1036E0000301B0930401ADCE803269F48091E8000B
:1036F00082FFFCCF67E085E091E00E94FB0C8BEF3E
:103700008093E8009ECE823209F09BCE8F89809311
:103710000C01EEEFFFE7859194918B3F9C4D51F1A9
:10372000E0E0F8E08091050190910601A091070189
:10373000B0910801803B9440A105B105F1F480915E
:103740000C0180FD1AC0EE3F8AE0F80789F587E793
:1037500097E791838083809160008093D40288E111
:103760009BE00FB6F894A895809360000FBE9093ED
:10377000600067CEEEEFFAE0D5CF80819181873788
:10378000974709F05ECEA89580916000886180938C
:1037900060008091D40280936000EE3F2AE0F2073F
:1037A00089F08091FE0A9091FF0A9183808349CE2F
:1037B000808191818737980751F29093FF0A809317
:1037C000FE0AC5CF1092FF0A1092FE0A3ACE0E945E
:1037D000E10BDC0112960D911C910115110509F404
:1037E000E8CED801ED91FC910190F081E02DBE0171
:1037F0006B5E7F4FC8010995811123CEF8010085CA
:103800001185EBCF181619060CF41BCED2CEF1E0C1
:10381000FF12BECE6CE27FE004CF1F920F920FB674
:103820000F9211242F933F938F939F93AF93BF9346
:103830008091C8029091C902A091CA02B091CB02B6
:103840003091C70223E0230F2D3758F50196A11DB3
:10385000B11D2093C7028093C8029093C902A09320
:10386000CA02B093CB028091CC029091CD02A0917C
:10387000CE02B091CF020196A11DB11D8093CC0262
:103880009093CD02A093CE02B093CF02BF91AF919F
:103890009F918F913F912F910F900FBE0F901F908E
:1038A000189526E8230F0296A11DB11DD2CFEF92E5
:1038B000FF920F931F93CF93DF93F82E192FE62ECD
:1038C000042F81E0860F880F0E94760C83E00E940F
:1038D000760CCF2DD12FEC0EFD2EF11CCE15DF0571
:1038E000B9F007FF13C0FE0184910E94760C182FD7
:1038F00080E00E94760C812321968111EFCFDF9129
:10390000CF911F910F91FF90EF9008958881EDCF97
:1039100081E0F5CFCF93DF931092E9061092E8068D
:1039200088EE93E0A0E0B0E08093EA069093EB0687
:10393000A093EC06B093ED0682E291E09093E70647
:103940008093E6068FEF9FEF9093F3068093F20645
:1039500010929B0710929A078CE491E0909399073C
:1039600080939807109291071092900780E491E05D
:1039700090938F0780938E0798E09093970781E04C
:1039800080939607109293071092940710929207D3
:1039900080939507109287071092860724E331E001
:1039A000309385072093840790938D0780938C072D
:1039B0001092890710928A071092880780938B07CC
:1039C000C4E5D7E0198218821B821A821D821C82EC
:1039D00050E040E06EEE71E0CE010E9406172696A0
:1039E00087E0C438D80771F7C6E3D7E01982188298
:1039F0001B821A821D821C8250E040E06EEE71E054
:103A0000CE010E940617269687E0C435D80771F7C5
:103A1000DF91CF910895CF93DF93CDB7DEB7609755
:103A20000FB6F894DEBF0FBECDBF789484B5826028
:103A300084BD84B5816084BD85B5826085BD85B552
:103A4000816085BD80916E00816080936E001092D0
:103A5000810080918100826080938100809181004B
:103A600081608093810080918000816080938000DC
:103A7000809191008260809391008091910081609B
:103A8000809391008091900081608093900080915C
:103A9000C10084608093C1008091C10082608093E6
:103AA000C1008091C10081608093C1008091C300FA
:103AB00081608093C3008091C00082608093C000C9
:103AC0008091C20081608093C20080917A008460FE
:103AD00080937A0080917A00826080937A0080914E
:103AE0007A00816080937A0080917A008068809368
:103AF0007A001092E5021092D5021092D7028091BE
:103B0000D70081608093D70080EA8093D80089B580
:103B1000806189BD89B5826089BD09B400FEFDCF91
:103B200061E070E080E090E00E942D0D8091D8006F
:103B30008F7C80618093D8008091E000807F8093AB
:103B4000E0008091E1008E7E8093E1008DE0809323
:103B5000E200559A209A0E94060F82E480930001A9
:103B6000809164008E7F8093640080917A008064ED
:103B700080937A0080917A0086FDFCCF00917800D6
:103B8000109179000E94080DAB01BC01C801B0E0A2
:103B9000A0E0DC01992788276C017D01C40ED51EA9
:103BA000E61EF71EC701B601209164002160209334
:103BB0006400611571058105910511F00E94892F3E
:103BC0001092C3021092C2021092C6020E94060F07
:103BD0000E945C0F80E80E94510F8823A9F05C9836
:103BE00085EA8EBD00000DB407FEFDCF5C9A2E98CD
:103BF0002F982D988091640080628093640081E00A
:103C000083BF889513BEFCCF84E00E94510F8823A8
:103C100009F448C02D9884E80E94510F8823E1F0F0
:103C20000E94F70E88EC90E00E94F90E2F9882E037
:103C300090E00E9427318F3F29F06FEF82E090E003
:103C40000E942F3184EF91E00E94F90E2F9A84E8B0
:103C50000E94510F8111FBCF84E10E94510F8823F4
:103C6000E1F00E94F70E88EC90E00E94F90E2E9889
:103C700082E090E00E942731882329F060E082E012
:103C800090E00E942F3184EF91E00E94F90E2E9A6D
:103C900084E10E94510F8111FBCF88EC90E00E94DB
:103CA000F90EB2CF0E94F70E82E090E00E94B915A3
:103CB000882309F441C03E9A3F9A81E090E00E9437
:103CC000B91581FF13C0082F0470302E82FD2E9885
:103CD00001EF1FEFB8E0AB2EB12C80E40E94510F32
:103CE000882369F12E9A2F9A0E94F70E82E390E0C2
:103CF0000E94F90E0E94FE0E8111F8CFE2E04E2ED6
:103D0000512C612C712C8FB7F8944091C8025091BE
:103D1000C9026091CA027091CB028FBF8091580294
:103D2000882309F4D0C01092580280E090E0892BDB
:103D300051F30E940000E7CF3E983F98BECF33205A
:103D400029F00430110511F42E9A2F9881E00E9479
:103D5000DC07980117FF04C022273327201B310BF3
:103D600027703327C80117FD0796A3E0959587951F
:103D7000AA95E1F717FF05C00197A501421B530B58
:103D80009A01BC017695762F6627779567956A51DB
:103D90007D4FF12CE12C2501421A530A8E3F5FEF33
:103DA000950709F43EC0DB0150E040E0F701E75C15
:103DB000F74F4F013B01F0E86F0E711C8F3F9807E2
:103DC00081F0F401E40FF51FE491022E01C0EE0F23
:103DD0000A94EAF75496FC915497EF2B5496EC937F
:103DE000549721153105B9F0F401E40FF51F249023
:103DF0006301C40ED51EE22DF0E0042C02C0F5953F
:103E0000E7950A94E2F7FE87ED87F6012488FD85A1
:103E10002F2AF601248A4F5F5F4F119648355105CE
:103E200069F60196F8E5EF0EF11C60587F4F40EB04
:103E3000E416F10409F0B2CF0E945C0F8FE090E02D
:103E40000E94F90E0F5F1F4F0931110509F045CF90
:103E5000332011F02F9A2D9880E991E00E94F90EFD
:103E60000E94F70E81E090E00E94B91580FF3ECFDE
:103E70008AE090E00E94B9159FEF980F9E3F08F0EE
:103E800035CF22E330E030935B0220935A0228E3DF
:103E900030E030935D0220935C020BE010E0682F6D
:103EA00088E997E00E94CA10C8010E94B9150F5F07
:103EB0001F4F0131110599F70E945C0F88EE93E0C6
:103EC0000E94F90E13CF80915902942F981B892FCD
:103ED00090910001891748F48F5F891708F025CF6A
:103EE00081E083BF889513BE20CF81E08093580284
:103EF00040935902809156029091570201969093F7
:103F000057028093560280915F0280935E020E9466
:103F1000FE0E80935F028091C6028111F5C0209150
:103F2000C2023091C302E6EEF2E081118FEF00246D
:103F300081938193819381930394D1F710925D02D1
:103F400010925C0210925B0210925A021092C5020B
:103F50001092C4022130310561F48091C002909129
:103F6000C1024F9734F087E190E09093C3028093B1
:103F7000C2028091C2029091C3028831910508F07B
:103F8000AEC4FC01EA53F04E0C94A633DE1F22208F
:103F9000F120CC20CC206D219621AF211422AD2020
:103FA0009F229F229F229F22AB22D7227422F62299
:103FB000F622992399239923992306244CE65EE05F
:103FC00070E060E090E080E00E94DD094CE65EE099
:103FD00070E060E082E690E00E94DD098AE290E015
:103FE00090935B0280935A028FE090E090935D0281
:103FF00080935C0263E67EE088E997E00E94A60E6B
:1040000087E680938907809388078AE380938A07ED
:104010006CE57EE084E897E00E94A60E6AE47EE00C
:1040200084E597E00E94771681E090E09093BF02CC
:104030008093BE021092BD021092BC0241E050E09B
:1040400060E04DC00E9468186091BA027091BB0296
:10405000CE0101960E94D716CE0101960E947213DE
:10406000CE0101960E94D61460E47EE084E597E0DC
:104070000E94771665E37EE08AE597E00E94771656
:104080006AE27EE080E697E00E94771666E27EE0D4
:1040900086E697E00E9477168091BA029091BB0263
:1040A000892B09F057C06BE17EE08CE697E00E9417
:1040B000771666E17EE082E797E00E94771686E059
:1040C00090E09093BF028093BE021092BD0281E007
:1040D0008093BC024091BE025091BF0261E080E03B
:1040E0000E94F40D2091BE023091BF0200E0409189
:1040F000BC026091BD028091C4029091C5020E94F1
:10410000561181E08093C602C090C202D090C302D3
:10411000B8E1CB16D10408F07CC4F601EE56FF4D91
:104120000C94A6338C248C248C248C248C248C24F6
:104130008C24682BDC2ADC2ADC2AE02AE02AE02A0C
:10414000DC2ADC2AE02A5E2C5E2C5E2C5E2C5E2CA7
:104150005E2CDC2A84E090E0B4CF0E9468186BE00B
:104160007EE0CE0101960E949F16CE0101960E942C
:104170007213CE0101960E94D61482EA92E00E9448
:104180008A174091BE025091BF026091BC0280919B
:10419000BD020E94F40DB5CF0E9468188091C20242
:1041A0009091C30261E07EE0039711F066EF7DE03D
:1041B000CE0101960E949F16CE0101960E947213B5
:1041C000CE0101960E94D6148AE892E00E948A17D6
:1041D0004091BE025091BF026091BC028091BD022D
:1041E0007FCF0E9468186CEE7DE0CE0107960E949A
:1041F0009F166091BA027091BB02CE0101960E9497
:10420000D716BE016F5F7F4FCE0107960E944616FC
:10421000CE0101960E94D6141A8219821C821B823A
:104220001E821D826F8178856115710531F04B8585
:104230005C85CE0101960E940617CE0101960E9470
:104240007213CE0101960E94D61474E5E72E77E032
:10425000F72E70E060E08B010F5F1F4F8091BA0274
:104260009091BB02681779070CF0B801CE01019656
:104270000E94D716BE016F5F7F4FC7010E94BB151A
:10428000CE0101960E94D614A6E0EA0EF11CB801F8
:104290000530110501F71093BF020093BE0281E0C3
:1042A0008093BD028093BC0245E050E061E00E9433
:1042B000F40D2091BE023091BF0200E04091BC029B
:1042C0006091BD028091C4029091C5020E94561176
:1042D000CE0107960E94D61414CF0E94681861EE92
:1042E0007DE0CE0101960E949F16CE0101960E94AC
:1042F0007213CE0101960E94D61466ED7DE084E52E
:1043000097E00E94771669EC7DE08AE597E00E94CD
:10431000771682E090E09093BF028093BE021092E5
:10432000BD021092BC0242E050E08ACE0E946818A2
:1043300064EC7DE0CE0101960E949F16CE010196AD
:104340000E947213CE0101960E94D61466EB7DE0A6
:1043500084E597E00E94771667EA7DE0D6CF68E9AA
:104360007DE086E397E00E9477166DE87DE08CE3C0
:1043700097E00E9477166091880270918902CE01C1
:1043800001960E943117BE016F5F7F4F8CE397E06B
:104390000E944616CE0101960E94D61467E87DE081
:1043A0008CE397E00E941C1666E77DE082E497E0CC
:1043B0000E94771668E67DE088E497E00E94771611
:1043C0006091860270918702CE0101960E9431179A
:1043D000BE016F5F7F4F88E497E00E944616CE01D2
:1043E00001960E94D61484E090E090938502809319
:1043F0008402109283020E94E31282E48093890770
:104400008093880787E380938A076FE97CE084E8DC
:1044100097E00E94A60E83E490E00E94211087E6B8
:1044200090E00E9421106DCE0E943A2F6B017C011A
:104430006FE87CE086E397E00E94771668E87CE00E
:104440008CE397E00E94771687E090E090938202D9
:104450008093810283E090E09093850280938402B0
:1044600010928302C701B601A30192010E943D315F
:10447000672B79F463E87CE08CE397E00E941C16DC
:104480006AE77CE082E497E00E9477160E94E312DC
:1044900038CE63E77CE08CE397E00E941C1669E667
:1044A0007CE082E497E00E947716809186029091EA
:1044B0008702039790938702809386021816190645
:1044C0002CF369E57CE088E497E00E94771684E0AD
:1044D00090E0909385028093840287E190E090932E
:1044E000820280938102D2CF66E57DE086E397E089
:1044F0000E94771668E47DE08CE397E00E947716CF
:1045000069E37DE082E497E00E9477166DE27DE04A
:1045100088E497E00E94771684E090E0909385020B
:1045200080938402109283020E94E3120E94CF12B1
:1045300081E090E09093820280938102E2CD0E941C
:10454000E3128091C2029091C3020A9709F4D9CD77
:104550000E94CF12D6CD64E571E086E397E00E9419
:10456000271767E671E08CE397E00E9427176CE756
:1045700071E082E497E00E94271760E971E088E427
:1045800097E00E94271762EA71E08EE497E00E94AC
:10459000271785E090E0909385028093840281E064
:1045A000809383020E94E3128FE090E0C3CF6EEE0F
:1045B00071E086E397E00E94271766EB71E08CE3D9
:1045C00097E00E94271765EC71E082E497E00E9473
:1045D000271783E090E090938502809384021092E5
:1045E00083020E94E31287E190E0A4CF66E27DE0BF
:1045F000419711F060E27DE086E397E00E94771634
:1046000060917F0270918002CE0101960E94A816EF
:10461000BE016F5F7F4F86E397E00E944616CE0192
:1046200001960E94D6146CE27DE08CE397E00E9434
:1046300077166BE27DE082E497E00E947716809126
:10464000C2029091C30261E17DE0419711F06BE0FD
:104650007DE088E497E00E94771667E17DE08EE4D4
:1046600097E00E94771685E090E090938502809312
:10467000840281E0809383020E94E312E0917F0232
:10468000F0918002EE0FFF1FEE0FFF1FE657FD4F68
:10469000208131814281538160913A0770913B07BB
:1046A000E5E0E69FC001E79F900D11246AE070E00D
:1046B0000F960E9467148091C2029091C3024197A5
:1046C000E9F420917B0230917C0240917D0250916F
:1046D0007E026EE270E087E390E00E9467140E9421
:1046E0008A1467E07DE0CE0101960E949F16CE01FC
:1046F00001960E943414CE010196ECCD87E380939D
:104700009307809392078EE280939407E0917F0253
:10471000F0918002EE0FFF1FEE0FFF1FEE55FD4FD1
:1047200040815181628173818EE897E00E94D913A4
:10473000D6CF6CEF7CE08331910559F06FEE7CE0D1
:104740008431910531F061EE7CE0459711F062ED26
:104750007CE086E397E00E94771666E07DE08CE3DC
:1047600097E00E94771665E07DE082E497E00E9482
:104770007716809181029091820261EC7CE005972E
:1047800011F069EB7CE088E497E00E94771669EC11
:104790007CE08EE497E00E94771685E090E09093AD
:1047A00085028093840281E0809383020E94E31259
:1047B00080918102909182020597F9F4209177020D
:1047C000309178024091790250917A0265E270E06E
:1047D00082E390E00E94671420917B0230917C027A
:1047E00040917D0250917E026EE270E087E390E09E
:1047F0000E94671465EB7CE076CF209173023091C4
:1048000074024091750250917602E0CF609173027C
:1048100070917402809175029091760200917B02F2
:1048200010917C0220917D0230917E02600F711FF9
:10483000821F931F009177021091780220917902D4
:1048400030917A02601B710B820B930B0E940A302D
:1048500020E030E04CEF51E40E9444320E944F339C
:104860000E94EC320E94B6326B016EEE71E086E37C
:1048700097E00E94271763ED71E08CE397E00E94B8
:10488000271760EE71E082E497E00E942717B601D7
:104890006536710514F064E670E0CE0101960E9461
:1048A0003117BE016F5F7F4F82E497E00E9446168A
:1048B000CE0101960E94D6146FEE71E088E497E075
:1048C0000E9427171092830284E090E09093850263
:1048D000809384021092820210928102D7CD85E0EB
:1048E00090E090935B0280935A0290935D028093D4
:1048F0005C026EEA7CE088E997E00E94A60E409197
:10490000C2025091C302052E000C660B770B88E99A
:1049100097E00E94D913F5CB80E80E94460F8111E1
:104920001AC080E10E94460F811115C080E20E94EA
:10493000460F811110C080E40E94460F81110BC008
:1049400088E00E94460F811106C084E00E94460F55
:10495000882309F45EC0A090BE02B090BF023090E0
:10496000BC02E090C402F090C50201E09501432D25
:104970006091BD02C7010E945611B5010B2C000CBD
:10498000880B990B0E940A3020E030E040E05FE3A2
:104990000E9469306D877E878F87988B20E030E09A
:1049A000A9010E94443320E030E040E05FE387FD4E
:1049B00033C06D857E858F8598890E94D8310E948D
:1049C000B6328B0188248394912CE616F7061CF0EE
:1049D00032E0832E912C80E10E94460F882359F10A
:1049E000EFEFEE1AFE0AEA14FB04ECF4F092C502B3
:1049F000E092C4022091BE023091BF0200E04091DB
:104A0000BC026091BD028091C4029091C5020E94D7
:104A100056110E945C0F89C96D857E858F859889A6
:104A20000E94D731CCCFF1E0AF1AB108B092C502E5
:104A3000A092C402DFCF80E80E94460F882371F065
:104A400001E0E01AF108F092C502E092C402F7FE1C
:104A5000D1CF1092C5021092C402CCCF80E40E9444
:104A6000460F8823D9F03320A9F08A94892891F43D
:104A7000E00EF11EF092C502E092C4028091C402E1
:104A80009091C5028A159B050CF4B4CF41E0A41A9D
:104A9000B108CCCF3FEFE31AF30AECCF80E20E94DB
:104AA000460F8823B9F0332089F052E0851691042F
:104AB00069F4E01AF10AF092C502E092C402809112
:104AC000C4029091C50297FF95CFC3CF81E0E81A49
:104AD000F108F1CF88E00E94460F882309F459C5F8
:104AE0001092C60293E0C916D10409F4BFC308F0BE
:104AF0005AC0B1E0CB16D10409F486C0E2E0CE166C
:104B0000D10409F4B0C0EF2809F074CF81E090E03F
:104B10009093C3028093C20220ED37E040E050E062
:104B200020937B0230937C0240937D0250937E025F
:104B300088E893E1A0E0B0E0809377029093780258
:104B4000A0937902B0937A021092730210927402C9
:104B500010927502109276021092BB021092BA0265
:104B6000109272021092710284E690E090937002AB
:104B700080936F0282E390E0909387028093860295
:104B8000E2EAF2E08AEB92E0119211921192119214
:104B90008E179F07C9F71092C1021092C00280E0E1
:104BA0000E94DE1427CFF5E0CF16D10409F47EC4AD
:104BB00008F423C416E0C116D10409F0A4CF86E09E
:104BC00090E0909382028093810210926B02109287
:104BD0006C0210926D0210926E02E114F10409F45D
:104BE000C9C4EA94EF2809F005CF86E190E09093DC
:104BF000C3028093C2028091730290917402A091CB
:104C00007502B091760221C4D0928202C0928102D4
:104C100092E0E916F104F1F074F4E114F104B9F052
:104C200084E090E0EA94EF2809F0E4CE9093C30288
:104C30008093C202DFCEE4E0EE16F10489F06CF05E
:104C400086E090E005E0E016F10481F3D3CE83E046
:104C500090E0ECCF89E090E0E9CF82E090E0E6CF11
:104C600085E090E0E3CF8091BA029091BB02E81614
:104C7000F9061CF01FEFE11AF10AF092BB02E09274
:104C8000BA0281E00E94DE140E943A2F24E130E053
:104C900040E050E00E943D319B0141E050E05093E4
:104CA00082024093810210928302FB013197E1312D
:104CB000F10508F0D6C2E15AF94D0C94A6337026DE
:104CC0009726B626E926E9261427142741278827A0
:104CD00088278827EA27EA273E285F288E28FE288B
:104CE00063ED7BE086E397E00E94771661EC7BE062
:104CF0008CE397E00E94771668EB7BE082E497E014
:104D00000E94771683E090E090938502809384025E
:104D100022E030E040E050E020939E0230939F027A
:104D20004093A0025093A1028AE090E07FCF67EA0F
:104D30007BE086E397E00E94771667E97BE08CE3EF
:104D400097E00E94771682E090E09093850280932E
:104D500084028AE790E0A0E0B0E08093960290930E
:104D60009702A0939802B0939902DECF66E87BE0A9
:104D700086E397E00E94771668E77BE08CE397E094
:104D80000E94771667E67BE082E497E00E94771640
:104D90006AE57BE088E497E00E94771684E090E083
:104DA00090938502809384020E943A2F2EE734E08C
:104DB00040E050E00E943D316E5A7C4F8F4F9F4F34
:104DC00060938E0270938F02809390029093910271
:104DD000ABCF6AE47BE086E397E00E9477166BE353
:104DE0007BE08CE397E00E9477166DE27BE082E443
:104DF00097E00E94771663E27BE088E497E00E94E8
:104E0000771684E090E090938502809384020E945C
:104E10003A2F29EA31E640E050E00E943D31605BE4
:104E2000794B8F4F9F4FCCCF64E17BE086E397E0D7
:104E30000E94771663E07BE08CE397E00E94771690
:104E400060EF7AE082E497E00E94771683E090E0DA
:104E500090938502809384020E943A2F21E63AEED5
:104E600040E050E00E943D316058774C8E4F9F4F9C
:104E700060938A0270938B0280938C0290938D02D0
:104E800053CF61EE7AE086E397E00E94771665EDF6
:104E90007AE08CE397E00E94771682E090E09093AE
:104EA00085028093840260917B0270917C028091E4
:104EB0007D0290917E020E940A3020E030E040E4C2
:104EC00050E40E9444326B017C0120E030E0A901F3
:104ED0000E94443320E030E040E05FE387FD13C0F0
:104EE000C701B6010E94D8310E94B632660F771F03
:104EF000881F991F60937B0270937C0280937D02D0
:104F000090937E0211CFC701B6010E94D731ECCF3A
:104F1000E2EAF2E04AEB52E090E080E0C190D1900A
:104F2000E190F1908C0D9D1D4E175F07B9F7C29768
:104F30000CF43FC382E090E02930310539F084E081
:104F400090E02A30310511F085E090E090938902DD
:104F50008093880269EC7AE086E397E00E947716F6
:104F600064EC7AE08CE397E00E9477166091880207
:104F70007091890261507109CE0101960E9431172A
:104F8000BE016F5F7F4F8CE397E00E944616CE0113
:104F900001960E94D6146CEB7AE08CE397E00E94B5
:104FA0001C1660EB7AE082E497E00E94771665EACF
:104FB0007AE088E497E00E94771684E090E090938E
:104FC00085028093840287E090E090938202809330
:104FD0008102AACE80917B0290917C02A0917D02F9
:104FE000B0917E02843F9140A105B1050CF4E1C26D
:104FF0000E949E1205970CF4DCC20E943A2F23E017
:1050000030E040E050E00E943D316B0166E97AE01B
:1050100086E397E00E947716F2E0CF16D104C8F439
:1050200069E77AE0CD2811F069E67AE08CE397E051
:105030000E94771669E87AE082E497E00E9477168A
:1050400083E090E090938502809384028BE090E06F
:10505000EDCD6BE57AE08CE397E00E9477166DE486
:105060007AE082E497E00E94771664E47AE088E4CC
:1050700097E00E94771684E090E0E4CF63E37AE063
:1050800086E397E00E94771663E27AE08CE397E08C
:105090000E94771661E17AE082E497E00E94771639
:1050A00060E07AE088E497E00E94771684E090E080
:1050B00090938502809384028DE090E0B7CD80913B
:1050C0007B0290917C02A0917D02B0917E028C3295
:1050D0009140A105B1050CF46CC26DEE79E086E358
:1050E00097E00E9477166DED79E08CE397E00E94DF
:1050F00077166EEC79E082E497E00E94771663EC15
:1051000079E088E497E00E94771684E090E090933D
:105110008502809384028CE090E088CD0E949E12EC
:1051200008970CF446C20E943A2F27E030E040E096
:1051300050E00E943D318B010F5F1F4F0E943A2FBC
:1051400026E030E040E050E00E943D316B01FB0181
:10515000EE0FFF1FEE0FFF1FEE55FD4FA801012EB2
:10516000000C660B770B80819181A281B381840F43
:10517000951FA61FB71F80839183A283B38368EB1B
:1051800079E086E397E00E947716B801CE01019698
:105190000E943117BE016F5F7F4F86E397E00E9448
:1051A0004616CE0101960E94D6146DEA79E08CE392
:1051B00097E00E947716B601CE0101960E94A816CC
:1051C000BE016F5F7F4F8CE397E00E944616CE01D1
:1051D00001960E94D6146DEF71E082E497E00E9480
:1051E00027176FE072E088E497E00E94271784E0B9
:1051F00090E0909385028093840296CD6DE172E0F9
:1052000086E397E00E9427176CE272E08CE397E058
:105210000E9427176EE372E082E497E00E9427174E
:105220006DE472E088E497E00E94271784E090E044
:1052300090938502809384020E943A2F27E232E005
:1052400040E050E00E943D3166507F4F8F4F9F4FAE
:1052500060939202709393028093940290939502CC
:1052600063CD5093C3024093C202C4CB0E949E12EE
:105270008C01D0928202C0928102F0928002E09270
:105280007F0218161906F4F163E57CE086E397E0E7
:105290000E94771662E57CE08CE397E00E94771627
:1052A00062E47CE082E497E00E9477166CE37CE0A5
:1052B00088E497E00E94771660917F0270918002E7
:1052C000CE0101960E94A816BE016F5F7F4F88E451
:1052D00097E00E944616CE0101960E94D6146AE31A
:1052E0007CE088E497E00E941C1684E090E09093B4
:1052F000850280938402109283028091C202909171
:10530000C30263CEF701EE0FFF1FEE0FFF1FE6573C
:10531000FD4FC080D180E280F38060917B0270916C
:105320007C0280917D0290917E026C157D058E0538
:105330009F0544F564E37CE086E397E00E947716DE
:1053400063E37CE08CE397E00E94771662E27CE006
:1053500082E497E00E94771660917F02709180024C
:10536000CE0101960E94A816BE016F5F7F4F88E4B0
:1053700097E00E94BB15CE0101960E94D61460E210
:105380007CE0AFCF21E130E03093C3022093C20232
:1053900010926B0210926C0210926D0210926E02CB
:1053A0000E940A304B015C01C701B6010E940A301D
:1053B0009B01AC01C501B4010E9444320E94EC3251
:1053C0000E94B63260936002709361028093620221
:1053D00090936302012E000C220B330B0617170764
:1053E000280739070CF006CB009360021093610286
:1053F0002093620230936302FDCA84E090E09093B0
:10540000820280938102F0928002E0927F02F70193
:10541000EE0FFF1FEE0FFF1FEE55FD4F80819181B4
:10542000A281B381181619061A061B06BCF422E1E4
:1054300030E03093C3022093C20210926B021092AC
:105440006C0210926D0210926E0280936002909333
:105450006102A0936202B0936302CCCA6AE17CE06D
:1054600086E397E00E94771669E17CE08CE397E0A1
:105470000E94771666E07CE082E497E00E9477164F
:1054800060917F0270918002CE0101960E94A81661
:10549000BE016F5F7F4F88E497E00E94BB15CE018D
:1054A00001960E94D61464E07CE01BCFD092820269
:1054B000C092810210926B0210926C0210926D02E7
:1054C00010926E02E114F10419F1EA94EF2809F048
:1054D00091CA80916A028823D1F168EF7BE086E36C
:1054E00097E00E94771669EE7BE08CE397E00E94DC
:1054F000771662EE7BE082E497E00E94771683E005
:1055000090E09093850280938402109283020CCCE9
:1055100083E190E09093C3028093C20240917B02AA
:1055200050917C0260917D0270917E0280917702A1
:1055300090917802A0917902B0917A0248175907A8
:105540006A077B070CF081CFDB01CA017ECF84E1C3
:1055500090E09093C3028093C20228E833E140E0D8
:1055600050E02093600230936102409362025093B6
:10557000630240CA85E190E09093C3028093C20227
:1055800080917B0290917C02A0917D02B0917E027D
:105590005CCF84E00E94460F882309F42BCA42E0C6
:1055A000C41AD10855E0C516D10408F023CA1092D8
:1055B000C60281E090E03ACB81E00E94B41229CA91
:1055C00080E00E94B412811124CA88E00E94460F34
:1055D000882309F41ECA1092C6028091C2029091DB
:1055E000C3028C30910509F44EC060F50B9709F0A9
:1055F00010CA80917102909172020196909372028A
:105600008093710280917B0290917C02A0917D0237
:10561000B0917E0280599140A109B10980937B022B
:1056200090937C02A0937D02B0937E0280916F02E2
:105630009091700205979093700280936F0281E0C1
:1056400090E041C08D309105E1F1409709F0E1C94A
:1056500080917B0290917C02A0917D02B0917E02AC
:10566000885E9340A109B10980937B0290937C02EC
:10567000A0937D02B0937E0282E390E09093870234
:1056800080938602DCCF80916F02909170020A961F
:105690009093700280936F0280917B0290917C02C4
:1056A000A0917D02B0917E02885C9109A109B109A7
:1056B00080937B0290937C02A0937D02B0937E0244
:1056C000BECF8EE090E09093C3028093C202A1C946
:1056D00084E00E94460F882309F440C01092C6025D
:1056E0000E943A2FA30192010E943D31672B682B43
:1056F000692BB9F46CE979E086E397E00E947716AC
:1057000061E979E08CE397E00E94771682E090E00F
:1057100090938502809384021092830281E090E04E
:1057200016C061E879E086E397E00E9477166BE7A0
:1057300079E08CE397E00E94771682E090E0909306
:105740008502809384021092830288E090E0909317
:105750008202809381028AE090E0B5CF88E00E94C7
:10576000460F882309F455C91092C6028091710230
:1057700090917202892BE9F46CE679E086E397E078
:105780000E9477166DE579E08CE397E00E9477162A
:1057900060E579E082E497E00E94771683E090E08C
:1057A00090938502809384021092830287E090E0B8
:1057B000CECF0E943A2FA30192010E943D31672B68
:1057C000682B692B49F46FE479E086E397E00E9447
:1057D00077166FE379E0ADCF8091880290918902CE
:1057E00001979093890280938802181619064CF449
:1057F0006EE379E086E397E00E9477166EE279E047
:1058000098CF0E943A2F23EE34E040E050E00E940F
:105810003D318B0102511D4F6CE179E086E397E049
:105820000E9477166EE079E08CE397E00E9477168D
:10583000B801CE0101960E943117BE016F5F7F4F04
:105840008CE397E00E944616CE0101960E94D61482
:105850006CEF78E082E497E00E94771669EE78E0DA
:1058600088E497E00E94771684E090E090938502A8
:105870008093840281E080938302012E000C220B2E
:10588000330B80917B0290917C02A0917D02B091BC
:105890007E02800F911FA21FB31F80937B02909303
:1058A0007C02A0937D02B0937E02803B9440A105D0
:1058B000B1050CF433CF80E190E049CF80E00E9445
:1058C000B4128111A6C888E00E94460F882309F40B
:1058D00039C18091C2029091C3028331910509F4CC
:1058E000B7C068F48131910509F479C04297C1F1DC
:1058F0001092C6028091810290918202E4CE85319D
:10590000910509F402C108F4CCC0469789F740918B
:105910006B0250916C0260916D0270916E028091E9
:10592000730290917402A0917502B0917602841B6B
:10593000950BA60BB70B8093730290937402A09300
:105940007502B093760280917B0290917C02A091C7
:105950007D02B0917E02840F951FA61FB71F36C02F
:1059600080917F029091800220916B0230916C02B5
:1059700040916D0250916E02880F991F880F991FF8
:10598000FC01EE55FD4FC080D180E280F380C21A49
:10599000D30AE40AF50AC082D182E282F3828657F2
:1059A0009D4FDC016D917D918D919C910E9496336C
:1059B00000917B0210917C0220917D0230917E0249
:1059C000DC01CB01800F911FA21FB31F80937B02CC
:1059D00090937C02A0937D02B0937E0289CF809148
:1059E0007F029091800220916B0230916C02409175
:1059F0006D0250916E02880F991F880F991FFC014C
:105A0000EE55FD4FC080D180E280F380C20ED31EE0
:105A1000E41EF51EC082D182E282F38286579D4F3A
:105A2000FC0160817181828193810E949633009193
:105A30007B0210917C0220917D0230917E026801F0
:105A40007901C61AD70AE80AF90AD701C601BECFFA
:105A500040916B0250916C0260916D0270916E02E8
:105A60008091770290917802A0917902B0917A02A8
:105A7000841B950BA60BB70B80937702909378024B
:105A8000A0937902B0937A0280917B0290917C027C
:105A9000A0917D02B0917E02841B950BA60BB70BE3
:105AA00095CF40916B0250916C0260916D027091A4
:105AB0006E028091770290917802A0917902B09164
:105AC0007A02840F951FA61FB71F809377029093C9
:105AD0007802A0937902B0937A0280917B02909130
:105AE0007C02A0917D02B0917E02840F951FA61FBB
:105AF000B71F80937B0290937C02A0937D02B093AA
:105B00007E0281E080936A02F3CE40916B02509155
:105B10006C0260916D0270916E028091730290919F
:105B20007402A0917502B0917602840F951FA61F92
:105B3000B71F8093730290937402A0937502B09381
:105B40007602A2CF8FB7F894C090C802D090C90255
:105B5000E090CA02F090CB028FBF8091C202909178
:105B6000C302419701E010E0029710F00AE010E054
:105B70008091660290916702A0916802B0916902DB
:105B8000B701A601481B590B6A0B7B0B809164027D
:105B900090916502823091050CF0F5C0453F51406F
:105BA0006105710510F40C94092501969093650226
:105BB0008093640280E80E94510F8823C1F1C09253
:105BC0006602D0926702E0926802F09269028091C8
:105BD000600290916102A0916202B0916302012E75
:105BE000000C220B330B40916B0250916C026091C0
:105BF0006D0270916E026C017D01C01AD10AE20A39
:105C0000F30AC416D506E606F7060CF447C0040FDF
:105C1000151F261F371F00936B0210936C022093F1
:105C20006D0230936E020E948A140C94092580E460
:105C30000E94510F882309F443C0C0926602D0929B
:105C40006702E0926802F09269024091600250910E
:105C5000610260916202709163022AE0209FC0019C
:105C6000219F900D1124092E000CAA0BBB0B009153
:105C70006B0210916C0220916D0230916E026A01EC
:105C80007B01C81AD90AEA0AFB0AC016D106E20645
:105C9000F3066CF0800F911FA21FB31F80936B025D
:105CA00090936C02A0936D02B0936E02BCCF4093B0
:105CB0006B0250936C0260936D0270936E02B3CFCF
:105CC00080E10E94510F882339F1C0926602D09280
:105CD0006702E0926802F0926902012E000C220B2A
:105CE000330B80916B0290916C02A0916D02B09188
:105CF0006E0280179107A207B3072CF0801B910B4F
:105D0000A20BB30BCBCF10926B0210926C021092CD
:105D10006D0210926E0287CF80E20E94510F88239D
:105D200021F1C0926602D0926702E0926802F0927E
:105D300069028AE0809FA001819F500D1124052EE9
:105D4000000C660B770B80916B0290916C02A09116
:105D50006D02B0916E0284179507A607B7079CF2F3
:105D6000841B950BA60BB70B99CF1092660210926D
:105D700067021092680210926902109265021092F6
:105D800064020C940925453651056105710508F03A
:105D900011CF0C940925CF93DF938EE497E00E94F6
:105DA000D61488E497E00E94D61482E497E00E941B
:105DB000D6148CE397E00E94D61486E397E00E9405
:105DC000D614C4E8D7E02697CE010E94D61487E007
:105DD000C435D807C1F7DF91CF9108958F929F9274
:105DE000AF92BF92CF92DF92EF92FF92CF93DF9369
:105DF000EC01688179818A819B816115710581053A
:105E0000910521F464E279ED8BE597E02DE133EF24
:105E100041E050E00E943D3149015A019B01AC0133
:105E2000A7EAB1E40E945C316B017C01ACEEB4EFF7
:105E3000A50194010E946A31C60ED71EE81EF91E04
:105E4000F7FE06C081E0C81AD108E10880E8F80A28
:105E5000C882D982EA82FB82C701B6019F77DF91AF
:105E6000CF91FF90EF90DF90CF90BF90AF909F9039
:105E70008F9008958F929F92AF92BF92CF92DF92B0
:105E8000EF92FF9260910D0170910E0180910F01D0
:105E900090911001611571058105910521F464E26D
:105EA00079ED8BE597E02DE133EF41E050E00E9482
:105EB0003D3149015A019B01AC01A7EAB1E40E94BE
:105EC0005C316B017C01ACEEB4EFA50194010E9442
:105ED0006A31C60ED71EE81EF91EF7FE06C081E025
:105EE000C81AD108E10880E8F80AC0920D01D092E2
:105EF0000E01E0920F01F0921001C701B6019F77E9
:105F0000FF90EF90DF90CF90BF90AF909F908F90D9
:105F1000089560930D0170930E0180930F0190938B
:105F200010010895FB01DC0105900D920020E1F7BE
:105F30000895FC0105900020E9F7809590958E0F5B
:105F40009F1F0895BB274A3031F4992322F4BDE204
:105F5000909581959F4F0C94DF2FBB272A3051F4E9
:105F6000992342F4BDE290958095709561957F4F9D
:105F70008F4F9F4F0C94BD2FBB27FA01A62F62179E
:105F8000710581059105330B30FB66F0AA27660F7A
:105F9000771F881F991FAA1FA21710F0A21B6395D5
:105FA0003850A9F7A05DAA3308F0A95DA19336F790
:105FB000B111B1931082CA010C94F82FBB27FB01D9
:105FC0005527AA27880F991FAA1FA41710F0A41BF2
:105FD00083955051B9F7A05DAA3308F0A95DA1934C
:105FE000009779F7B111B1931192CB010C94F82F6E
:105FF000DC01FC01672F71917723E1F7329704C030
:106000007C916D9370836291AE17BF07C8F30895BA
:10601000E89409C097FB3EF4909580957095619542
:106020007F4F8F4F9F4F9923A9F0F92F96E9BB27F8
:106030009395F695879577956795B795F111F8CF74
:10604000FAF4BB0F11F460FF1BC06F5F7F4F8F4FDF
:106050009F4F16C0882311F096E911C0772321F0D5
:106060009EE8872F762F05C0662371F096E8862F6D
:1060700070E060E02AF09A95660F771F881FDAF7C4
:10608000880F9695879597F90895990F0008550FF1
:10609000AA0BE0E8FEEF16161706E807F907C0F0AE
:1060A00012161306E407F50798F0621B730B840BB6
:1060B000950B39F40A2661F0232B242B252B21F490
:1060C00008950A2609F4A140A6958FEF811D811D30
:1060D00008950E947C300C94ED300E94DF3038F03F
:1060E0000E94E63020F0952311F00C94D6300C94E9
:1060F000DC3011240C9421310E94FE3070F3959F06
:10610000C1F3950F50E0551F629FF001729FBB27AE
:10611000F00DB11D639FAA27F00DB11DAA1F649F4A
:106120006627B00DA11D661F829F2227B00DA11DFD
:10613000621F739FB00DA11D621F839FA00D611D83
:10614000221F749F3327A00D611D231F849F600DA4
:10615000211D822F762F6A2F11249F5750409AF0CD
:10616000F1F088234AF0EE0FFF1FBB1F661F771F59
:10617000881F91505040A9F79E3F510580F00C9424
:10618000D6300C9421315F3FE4F3983ED4F38695EA
:1061900077956795B795F795E7959F5FC1F7FE2BC4
:1061A000880F911D9695879597F9089597F99F67A0
:1061B00080E870E060E008959FEF80EC089500248F
:1061C0000A941616170618060906089500240A945C
:1061D00012161306140605060895092E0394000CE2
:1061E00011F4882352F0BB0F40F4BF2B11F460FF71
:1061F00004C06F5F7F4F8F4F9F4F089557FD90589A
:10620000440F551F59F05F3F71F04795880F97FB7A
:10621000991F61F09F3F79F0879508951216130634
:106220001406551FF2CF4695F1DF08C01616170663
:106230001806991FF1CF8695710561050894089598
:10624000E894BB2766277727CB0197F90895F9993A
:10625000FECF92BD81BDF89A992780B50895262F6B
:10626000F999FECF1FBA92BD81BD20BD0FB6F8943B
:10627000FA9AF99A0FBE01960895052E97FB1EF41F
:1062800000940E94543157FD07D00E94A63107FCAC
:1062900003D04EF40C94543150954095309521958F
:1062A0003F4F4F4F5F4F0895909580957095619542
:1062B0007F4F8F4F9F4F08950E94C831A59F900D2B
:1062C000B49F900DA49F800D911D11240895B7FFD8
:1062D0000C945C310E945C31821B930B08952F92C9
:1062E0003F924F925F926F927F928F929F92AF9266
:1062F000BF92CF92DF92EF92FF920F931F93CF93B3
:10630000DF93CDB7DEB7CA1BDB0B0FB6F894DEBF49
:106310000FBECDBF09942A88398848885F846E846F
:106320007D848C849B84AA84B984C884DF80EE80B9
:10633000FD800C811B81AA81B981CE0FD11D0FB6C2
:10634000F894DEBF0FBECDBFED010895A1E21A2E75
:10635000AA1BBB1BFD010DC0AA1FBB1FEE1FFF1F09
:10636000A217B307E407F50720F0A21BB30BE40B59
:10637000F50B661F771F881F991F1A9469F76095A0
:106380007095809590959B01AC01BD01CF0108955A
:10639000A29FB001B39FC001A39F700D811D112466
:1063A000911DB29F700D811D1124911D08955058AB
:1063B000BB27AA270E94EF310C94ED300E94DF30FA
:1063C00038F00E94E63020F039F49F3F19F426F4AB
:1063D0000C94DC300EF4E095E7FB0C94D630E92FFA
:1063E0000E94FE3058F3BA176207730784079507B7
:1063F00020F079F4A6F50C9420310EF4E0950B2EE4
:10640000BA2FA02D0B01B90190010C01CA01A00106
:106410001124FF27591B99F0593F50F4503E68F161
:106420001A16F040A22F232F342F4427585FF3CFA2
:10643000469537952795A795F0405395C9F77EF473
:106440001F16BA0B620B730B840BBAF09150A1F0BC
:10645000FF0FBB1F661F771F881FC2F70EC0BA0F42
:10646000621F731F841F48F4879577956795B795CA
:10647000F7959E3F08F0B0CF9395880F08F09927C5
:10648000EE0F9795879508950E9458320C94ED3041
:106490000E94E63058F00E94DF3040F029F45F3F60
:1064A00029F00C94D63051110C9421310C94DC302D
:1064B0000E94FE3068F39923B1F3552391F3951BA5
:1064C000550BBB27AA2762177307840738F09F5F15
:1064D0005F4F220F331F441FAA1FA9F335D00E2E82
:1064E0003AF0E0E832D091505040E695001CCAF7EF
:1064F0002BD0FE2F29D0660F771F881FBB1F2617B2
:1065000037074807AB07B0E809F0BB0B802DBF0188
:10651000FF2793585F4F3AF09E3F510578F00C9457
:10652000D6300C9421315F3FE4F3983ED4F3869546
:1065300077956795B795F7959F5FC9F7880F911D78
:106540009695879597F90895E1E0660F771F881F64
:10655000BB1F621773078407BA0720F0621B730B17
:10656000840BBA0BEE1F88F7E09508950E94BD32A8
:106570006894B1110C94213108950E94063188F07D
:106580009F5798F0B92F9927B751B0F0E1F0660FF7
:10659000771F881F991F1AF0BA95C9F714C0B13038
:1065A00091F00E942031B1E008950C942031672FC2
:1065B000782F8827B85F39F0B93FCCF38695779567
:1065C0006795B395D9F73EF4909580957095619550
:1065D0007F4F8F4F9F4F08950E942C3390F09F372D
:1065E00048F4911116F00C94213160E070E080E8DD
:1065F0009FEB089526F41B16611D711D811D0C94DF
:1066000003330C941E33882371F4772321F09850C0
:10661000872B762F07C0662311F499270DC0905160
:10662000862B70E060E02AF09A95660F771F881F2E
:10663000DAF7880F9695879597F908959F3F31F07F
:10664000915020F4879577956795B795880F911DA0
:106650009695879597F908950E940631A0F0BEE7B8
:10666000B91788F4BB279F3860F41616B11D672F41
:10667000782F8827985FF7CF869577956795B11D16
:1066800093959639C8F308950E94453008F48FEF2A
:10669000089519F416F40C94DC300C941E330E9407
:1066A0000631B8F39923C9F3B6F39F57550B87FF0B
:1066B0000E948F330024A0E640EA9001805856954E
:1066C000979528F4805C660F771F881F20F02617A7
:1066D0003707480730F4621B730B840B20293129DC
:1066E0004A2BA69517940794202531254A2758F759
:1066F000660F771F881F20F026173707480730F4EA
:10670000620B730B840B200D311D411DA09581F789
:10671000B901842F9158880F9695879508959150C7
:106720005040660F771F881FD2F70895DB018F93C3
:106730009F930E945C31BF91AF91A29F800D911DEC
:10674000A39F900DB29F900D11240895EE0FFF1F8F
:106750000590F491E02D09940F931F93CF93DF934D
:106760008230910510F482E090E0E0919E07F09174
:106770009F0730E020E0B0E0A0E0309799F42115C9
:10678000310509F44AC0281B390B24303105D8F5EE
:106790008A819B816115710589F1FB019383828355
:1067A000FE0111C0408151810281138148175907B0
:1067B000E0F04817590799F4109761F012960C937E
:1067C000129713961C933296CF01DF91CF911F91B0
:1067D0000F91089500939E0710939F07F4CF211502
:1067E000310551F04217530738F0A901DB019A0136
:1067F000BD01DF01F801C1CFEF01F9CF90939F07F1
:1068000080939E07CDCFFE01E20FF31F81939193FA
:106810002250310939832883D7CF20919C073091AA
:106820009D07232B41F420911301309114013093E3
:106830009D0720939C072091110130911201211591
:10684000310541F42DB73EB7409115015091160125
:10685000241B350BE0919C07F0919D07E217F3078D
:10686000A0F42E1B3F0B2817390778F0AC014E5FC0
:106870005F4F2417350748F04E0F5F1F50939D0759
:1068800040939C07819391939FCFF0E0E0E09CCFF1
:10689000CF93DF930097E9F0FC01329713821282C5
:1068A000A0919E07B0919F07ED0130E020E0109786
:1068B000A1F420813181820F931F20919C07309198
:1068C0009D072817390709F061C0F0939D07E093F1
:1068D0009C07DF91CF910895EA01CE17DF07E8F515
:1068E0004A815B819E0141155105B1F7E901FB83A6
:1068F000EA8349915991C40FD51FEC17FD0761F444
:10690000808191810296840F951FE9019983888384
:10691000828193819B838A83F0E0E0E012968D91DF
:106920009C9113970097B9F52D913C911197CD014A
:106930000296820F931F20919C0730919D07281784
:10694000390739F6309751F510929F0710929E073C
:10695000B0939D07A0939C07BCCFD383C283408193
:106960005181840F951FC817D90761F44E5F5F4F9F
:1069700088819981480F591F518340838A819B8167
:10698000938382832115310509F0B0CFF0939F07DF
:10699000E0939E079ECFFD01DC01C0CF13821282DF
:1069A000D7CFB0E0A0E0E7EDF4E30C9471318C01B7
:1069B000009751F4CB010E94AC338C01C801CDB7D4
:1069C000DEB7E0E10C948D31FC01E60FF71F9C016E
:1069D00022503109E217F30708F49DC0D901CD9187
:1069E000DC911197C617D70798F0C530D10530F361
:1069F000CE0104978617970708F3C61BD70B22977B
:106A0000C193D1936D937C93CF010E944834D6CF2C
:106A10005B01AC1ABD0A4C018C0E9D1EA0919E0715
:106A2000B0919F07512C412CF12CE12C109731F59E
:106A300080919C0790919D078815990509F05CC08D
:106A40004616570608F058C0809111019091120126
:106A5000009741F48DB79EB74091150150911601F2
:106A6000841B950BE817F90708F055C0F0939D07B4
:106A7000E0939C07F90171836083A0CF8D919C9175
:106A8000119712966C90129713967C901397A815F5
:106A9000B90559F56C0142E0C40ED11CCA14DB04DF
:106AA00020F1AC014A195B09DA011296159780F0C2
:106AB0006282738251834083D9016D937C93E11488
:106AC000F10471F0D7011396FC93EE93129776CFF1
:106AD00022968C0F9D1FF90191838083F301EFCFE4
:106AE000F0939F07E0939E0769CF4816590608F474
:106AF0002C017D01D3019ACFCB010E94AC337C01E4
:106B0000009749F0AE01B8010E948E35C8010E947D
:106B10004834870153CF10E000E050CFFB01DC0187
:106B200002C001900D9241505040D8F70895FB01EA
:106B3000DC0101900D920020E1F7089517E0C1EB10
:106B4000D7E004C0FE010E94A6332196C23BD107C4
:066B5000C9F7F894FFCF25
:106B560010FFFFFFFF00E100000000000001000041
:106B6600000000A007800000C18081000000000036
:106B76000000F50B600D160C0B0C5C0C1A0C380C97
:106B8600000000005012CA0E7D13E50D0000000043
:106B96000212CA0E7D13E50D00000000CA10CA0ECF
:106BA6007D13E50D596F7520656174206974206148
:106BB6006C6C2062757400666F7267657420746F02
:106BC60020627275736820796F75720074656574DA
:106BD600682E205468657920616C6C20726F740091
:106BE600616E6420796F752063616E27742065611C
:106BF6007400736F6C696420666F6F6420616E79D0
:106C06006D6F72652E002020204A757374207361A3
:106C160079206E6F0020202020746F2063616E64DF
:106C2600792E00202047616D65206F766572210000
:106C36002020596F75722073636F72653A200020A9
:106C4600206F7574206F66203130302E00696E20FB
:106C560061206C756E636820626F7820696E0074BF
:106C66006865207375627761792121210054686512
:106C7600206D61726B657420686173006265656E74
:106C860020666C6F6F64656420776974680063685A
:106C960065617020686F6D656D6164650041657240
:066CA6006F2121212100F5
:00000001FF
